:0600000076EF06F012008D
:0600080004EF08F01200F5
:100018000CEF08F012001DEE00F02DEE00F0F86A6B
:0600280092EF06F0120049
:1000300000003E0E006E016AFC0E026E036A046A46
:10004000076808680968066A1200D9CFE6FFE1CFA1
:10005000D9FFE65204501EE1040108BF1AD0400E39
:10006000E66E600EE66E000EE66E38EC06F0E552C7
:10007000E552E552010E046EDF6A400EDF5C09E2D4
:10008000DF50EA6AA00FE96E000EEA22EF6ADF2A6B
:10009000F4D717D100016051080A01E10DD10F0A10
:1000A00001E1D3D0010A01E1CAD0030A67E0010AE5
:1000B00058E0070A44E0010A01E003D10001020E02
:1000C000A06F00013A0EA16F0001010EA26F0001A6
:1000D000010EA36F0001A46B100EA56FA66BA76B9A
:1000E00001C0A8F002C0A9F003C0AAF0100E0001E0
:1000F000A95F000E0001AA5B0001AB6B0001030EBB
:10010000AC6F0001F80EAD6FAE69AF6BB06B000164
:10011000080EB16FB26BB36BB46B0001B56904012B
:100120000CBF0CD0400EE66EA00EE66E000EE66E22
:1001300008EC06F0E552E552E552046AC2D000012F
:10014000615107E13F0E006EF80E016E0268036A0E
:1001500006D03E0E006E016AFC0E026E036A046A4F
:10016000B0D0040E056E0028055C06E20400AED88F
:100170009DEC04F0052AF7D7046AA3D0E8680718B5
:1001800005E1E868081802E1E868091806E161C0BD
:1001900007F062C008F063C009F007500001611960
:1001A00008E108500001621904E1095000016319D7
:1001B00000E143E1DF6A00016551DF5C3EE2000ED1
:1001C000075C100E0858000E09582CE300285B6EDF
:1001D0005C6A0A0ED8905B365C36E806FBE15D6A25
:1001E0005CBE5D685B50075C5C5008585D50095808
:1001F00019E23A0E0001D8806555DF24EA6A660FDD
:10020000E96E000EEA22EF50E66E0650E96EEA6AE9
:10021000E9BEEA680A0EE926000EEA22E552E75036
:10022000EF6E062A072A000E0822000E09223A0E57
:10023000065C01E15ED8DF2ABED7046A42D059D8F5
:10024000076808680968046A3CD00001070EA06FBF
:1002500061C0A1F062C0A2F063C0A3F064C0A4F0CA
:1002600065C0A5F061C0F6FF62C0F7FF63C0F8FF8C
:10027000DF6A00016551DF5C0FE209003A0E000100
:10028000D8806555DF24EA6AA60FE96E000EEA22DF
:10029000F5CFEFFFDF2AEDD704010CBF0CD0400EE5
:1002A000E66EA00EE66E000EE66E08EC06F0E55275
:1002B000E552E552046A05D06592656A68D8FF0088
:1002C00000D0E552E552E7CFD9FF1200F66A05509B
:1002D000F76EF86AD890F736F836F736F836140E17
:1002E000A66EF29E550EA76EAA0EA76EA682A694C3
:1002F0001200D9CFE6FFE1CFD9FFE652DF6A000E48
:10030000E76E0618E8AE02D0063403D0E750D88076
:10031000065436E206505B6E5C6A5D6A5BAE02D0E4
:100320005C685D685B50075CF66E5C500858F76E61
:100330005D500958F86EDF50EA6A0A0FE96E000E48
:10034000EA22EF50F56E0D00DF2A0606065009E09E
:10035000DF50EA6A0A0FE96E000EEA22EF50F56EEE
:1003600001D0F5680C00DF2A240EA66EF29E550E11
:10037000A76EAA0EA76EA682065001E00606BFD79A
:10038000A694066AE552E552E7CFD9FF1200D9CF0D
:10039000E6FFE1CFD9FFE652DF6AFF0EDF5C0AE23B
:1003A000E868E85005E0E80600D000D000D0F9D7B2
:1003B000DF2AF3D7E552E552E7CFD9FF12005FD924
:1003C000E652645032E16296040100513C0BE8426F
:1003D000E8420D0828E1180E021923E1040E031962
:1003E00020E1100E026F040E036FDF6ADF505B6EB8
:1003F0005C6A080E5B5C000E5C5813E2DF50EA6A30
:10040000180FE96E040EEA22EF50E66EDF50EA6A3A
:10041000100FE96E040EEA22E552E750EF6EDF2A74
:10042000E5D70ED80AD03DD808D0040E645C03E1AD
:1004300062964DD802D0000E01D0010EE55224D1B3
:100440001ED9E652040104BF046B556A516A526A10
:10045000536A546A4FEC03F0DF6ADF505B6E5C6AEC
:10046000010E5B5C000E5C5819E2525017E1F76A0E
:10047000DF34FE0BF736F66EA40EF6260E0EF722CC
:100480000900F5CF5BF00800F5CF5CF004D05CC04C
:10049000FAFF5B50F96EFBDFDF2ADFD79ED8E5520B
:1004A000F3D0020E515C0EE176D80401180E026FF3
:1004B000040E036F080E016F00BD02D0C80E05D0F8
:1004C000880E03D0BCD8CCD88C0E006F1200040E5E
:1004D000575C0AE112C438FF0F013851000802E2EC
:1004E000050E01D0030E576E51040FE110D8020E15
:1004F000555C03E10401840E06D0040104BD02D062
:10050000C80E01D0880E046F12001FEF03F0B7D899
:10051000020EE126080E535C000E54580DE253C043
:10052000DEFF54C0DDFF555002E1010E03D055043B
:1005300006E1020E556E03D0080EDE6EDD6A040180
:1005400004930491010EDB500413DFCF05F4DE5059
:10055000535EDD50545A0001180EE26F040EE36F33
:1005600058A20CD085D810E0E0C0F6FFE1C0F7FF3C
:100570000800F55068D8F6E2DB06F4D779D804E035
:1005800087D8FCE2DB06FAD7020EE15C02E2E16A00
:10059000E552E16E79D073D8020EE126030E040114
:1005A0000015E76E010EE7CFDBFF01C4DFFFDE5071
:1005B0005326DD5054220001180EE06F040EE16F47
:1005C00057D804E065D8FCE2DB06FAD7020EE15CFE
:1005D00002E2E16AE552E16E57D06598525005E1BA
:1005E0003FD8840E006F040118D0040110AF17D05B
:1005F0005350165D5450175904E216C453F017C4F3
:1006000054F085DF010E516E2BD8800E006F04016F
:10061000180E066F040E076FC80E046F1200020E4C
:10062000516E0401056BC80E046F0401080E016FC2
:10063000180E026F040E036FC80E006F1200516A8D
:100640000401046B1200E2C0E9FFE3C0EAFFEF6EB1
:10065000E22B000EE323E02BE123DF06010E120064
:100660000401080E016F100E026F040E036F1200DA
:10067000D9CFE9FFDACFEAFFEE50ED101200D9CF63
:10068000E6FFE1CFD9FF1200E552E7CFD9FF120014
:10069000E0C0E9FFE1C0EAFFEF5023EF03F00401FF
:1006A0001051600BE842E842E842E842E8420009A3
:1006B00001E012001151070A43E00B0A41E0070A6A
:1006C00034E0010A24E00B0A20E0020A1EE0030ADB
:1006D0001AE0080A10E0010A0CE00F0A08E0030A19
:1006E00001E01200010E526E040E576E1200A1EFCF
:1006F00003F0D7EF03F0010E526E0001590EE06FC8
:10070000000EE16F0ED0F1EF03F01FEF04F0010EC9
:10071000526E14510001E06FE16B5A0EE027000E9B
:10072000E1235892010E536E1200010E526E1451C5
:10073000EA6A5A0FE96E000EEA2212C4EFFF1200B5
:100740001200800E0401105D31E11351030A20E014
:10075000010A0BE0030A29E1010E526E0001E40ECA
:10076000E06F0D0EE16F120E1ED0AAD89A0EF6267B
:100770000E0EB8D8020E0001F76AE025F66EE151C0
:10078000F7220900F5CF53F00A00F5CF54F00DD051
:1007900097D89E0EF6260E0EA5D8E0C0F6FFE1C053
:1007A000F7FF0800F550536E546A58821200010E8C
:1007B000526E0F0EE66E270EE66E0F0E9BD8010EE0
:1007C000E66E5A0EE66E000E95D812C459F004017A
:1007D000125103E1050E576E1200060E576EF3EF2D
:1007E00005F00401186B196B040110511F0B020A6C
:1007F0000EE0030A09E0010A17E1010E526E58A04B
:1008000013D00401188310D0010E526E0DD04AD8B7
:1008100001E0010E5ED8E2C0E9FFEA6EEF50040B82
:1008200003E00401010E186F520408E10001180EE4
:10083000E06F040EE16F5892020E536E1200040135
:1008400012050CE110511F0B000908E1010E526E58
:10085000030E115D02E1588001D05890125121E140
:1008600010511F0B02081DE114510F0B000919E074
:1008700019D801E0010E2DD8030E0401115D02E12B
:10088000840E03D014AF07D0400EE2C0E9FFE3C0EE
:10089000EAFFEF6E1200880EE2C0E9FFE3C0EAFF54
:1008A000EF6E1200010E526E14510F0B080DF35033
:1008B0005C6A000F5B6E040E5C221451800B120008
:1008C000010E526E1251F66EF76AD890F636F73670
:1008D0001200040DF35000015B24E26F000E5C2057
:1008E000E36F1200F7220900F5CFE0F00A00F5CF20
:1008F000E1F01200E66E76EC05F0E552E552E552C5
:10090000120065A60CD8570409E165BA07D0626ADF
:100910000F01366B36813689020E576E1200656AFA
:100920000F01366B6586010E576E1200656A0F0166
:10093000366B576A120096EF04F0575001E112002F
:100940006250040B05E00F013651040B01E083D81F
:1009500065B212006250010B05E00F013651010B28
:1009600001E093D86250100B05E00F013651100BD7
:1009700001E01FD86250200B05E00F013651200B1B
:1009800001E071D8030E575C01E21200566A040EB2
:10099000565C0EE26250080B0BE00F013651080B5B
:1009A00007E0DFEC01F0000901E16296562AEFD77B
:1009B0001200D9CFE6FFE1CFD9FF020EE12636CFF4
:1009C000DFFF0F01040E366F629865828C50040BB6
:1009D00001E0010E5B6E8C50080B01E0010E5B1014
:1009E000E76E010EE7CFDBFF8C968C94A198A08870
:1009F0000300A150100B05E1D050080B02E10300E9
:100A0000F8D7A098DF500F013613010EDB50E8B085
:100A10008C86E8A08C96010EDB50E8B08C84E8A0B0
:100A20008C94D50E4F6E020E506E4FC05BF050C0CE
:100A30005CF04F06000E505A5B505C1002E0040060
:100A4000F4D7020EE15C02E2E16AE552E16EE552A2
:100A5000E7CFD9FF120065920F01369562A402D04C
:100A60006294FCD712000F0126A10DD0800E040164
:100A7000005D07E1840E0401045D03E104018C0EB6
:100A8000006F0F012691629A1200636A626A0F0179
:100A90009F0E376F0F017B0E366F0F01386B0F0EF5
:100AA000E66E270EE66E0F0EE66E20D8E552E55292
:100AB000E5520F01160E266F62A605D0629600D091
:100AC00000D00000F9D765981FEC03F00401080E70
:100AD000016F0401100E026F040E036F04018C0EEF
:100AE000006F5890596A030E576E1200D9CFE6FF77
:100AF000E1CFD9FFFD0EDBCFE9FFFE0EDBCFEAFF32
:100B0000FC0EDB5004E0EE6AFC0EDB06F9D7E55282
:100B1000E7CFD9FF1200040110511F0B010801E0BB
:100B20001200145101E01200060E115D21E1135173
:100B3000230A1DE0010A0DE0030A19E1020E526EBC
:100B4000590405E10001080EE06F0E0EE16F090E79
:100B50000CD0020E526E590405E100017D0EE06FCB
:100B60000E0EE16F590403E11D0E536E546A588254
:100B700004011051600BE842E842E842E842E842D2
:100B8000010801E0120011510B0A26E0080A19E0E1
:100B9000090A12E0080A09E00B0A05E0080A01E068
:100BA0001200F1EF05F0F2EF05F0020E526E0001B7
:100BB0004A0EE06F000E0BD0020E526E13C44AF0C4
:100BC0001200020E526E00014B0EE06F000EE16F3C
:100BD0005892010E536E1200020E526E12C44BF068
:100BE0001200120012004C6A0F011E0E276F040142
:100BF000400E096F200E0A6F040E0B6F880E086FEF
:100C00000401600E0E6F040E0F6F400E0C6F120089
:100C1000D9CFE6FFE1CFD9FFE652FC0EDB5040080A
:100C200005E2400EF36EFC0EF3CFDBFFDF6AFC0E35
:100C3000DB50DF5C0FE2DF504DD8EF50E66EDF5047
:100C4000EA6A600FE96E040EEA22E552E750EF6EA1
:100C5000DF2AEDD7FC0EDBCF0DF4400E04010C179C
:100C60000C7D880E0C13E552E552E7CFD9FF120038
:100C7000D9CFE6FFE1CFD9FF4C6A040108BF25D0E8
:100C8000FC0EDBCF5BF00951D8805B5403E2FC0E15
:100C900009C4DBFF4C6AFC0EDB504C5C0FE24C508D
:100CA000EA6A200FE96E040EEA22EF50E66E4C501D
:100CB00011D8E552E750EF6E4C2AEDD70401400EF3
:100CC000096F0817087D880E08134C50E552E7CFCE
:100CD000D9FF1200E76EFD0EDBCFE9FFFE0EDBCF82
:100CE000EAFFE750E926000EEA2212001DEE00F0AE
:100CF0002DEE00F0F86AF66A100EF76E0800F55057
:100D0000FF0808E1010EF66E100EF76E0800F550B0
:100D1000FF0806E080AE02D000EF08F080AEFED7FC
:100D200001D812000DD8040034D837D8060E575C0D
:100D300005E16550020B02E125EC00F0F4D712004A
:100D4000600ED36E9B8C580E4F6E020E506E4FC0CD
:100D50005BF050C05CF04F06000E505A5B505C10C8
:100D6000F6E165A604D06592656AC7EC01F00F0153
:100D7000140E396F576A586A596A19EC00F04D6AB7
:100D80004E6A8C968C94959695940F01486B496B9E
:100D9000120081EC04F09DEF04F04D504E1004E180
:100DA000100E4D6E270E4E6E4D06000E4E5A060E5C
:100DB000575C02E28C868C94060E575C12E14D5013
:100DC0004E100FE10001E65102E18C868C94030E77
:100DD000E65D02E18C968C84E62BE651030801E285
:100DE000E66B12001201000200000008D8043C006B
:100DF00002000102000109022900010100C03209BC
:100E00000400000203000000092111010001221D5D
:100E100000070581034000010705010340000104AC
:100E200003090434034D006900630072006F00631E
:100E300000680069007000200054006500630068CD
:100E4000006E006F006C006F0067007900200049A1
:100E5000006E0063002E0026034800490044002075
:100E600000550053004200200042006F006F0074E4
:100E7000006C006F0061006400650072000600FFF6
:100E80000901A10119012940150026FF00750895E7
:100E9000408100190129409100C0F60DF60D1F0E8A
:100EA000230E570E160BC00EF36E00EE00F00E0E62
:100EB00001D81200EA6002D0EE6AFCD7F350E96074
:060EC0001200EE6AFCD7EF
:06100000CBEF56F01200D8
:061008003EEF35F012007E
:0610180068EF24F0120055
:10102A000200FAAD000000050000E1000000F8AD82
:10103A000000FB02000002000000020100000000A4
:10104A0000013200000000000180004D0000000293
:10105A000000000000000132000000000001A700AB
:10106A00FBFFDFFF015700EFFF0400014E00F2FF14
:10107A000700014C00F3FF0800014A00F5FF0A00CF
:10108A00014400F8FF0B00014800FAFF0D00014E71
:10109A0000FCFF0F00015000FFFF100001320000AA
:1010AA00000A00012E000200090001330002000AB2
:1010BA0000012D0004000800012D000400080001B1
:1010CA002F000500080001310007000700012E006B
:1010DA00070006000132000800060001330009007B
:1010EA0005000136000A0004000134000A0003006A
:1010FA000139000B000300013D000C000200014110
:10110A00000D0001000146000E0001000146000E1C
:10111A0000FFFF0141000D00FFFF013D000C00FE32
:10112A00FF013E000C00FDFF0139000B00FDFF012D
:10113A0036000A00FCFF0133000900FBFF01320000
:10114A000800FAFF0135000800F9FF012E00060029
:10115A00F9FF012E000600F9FF012D000400F8FF37
:10116A00012D000400F8FF012E000200F7FF012EF6
:10117A00000200F7FF0132000000F6FF012D000017
:10118A0000F7FF012E00FEFFF7FF012900FEFFF81E
:10119A00FF012B00FDFFF8FF012F00FBFFF8FF0105
:1011AA002B00FBFFF9FF013100F9FFF9FF012E00C7
:1011BA00F9FFFAFF013200F8FFFAFF013300F7FFE7
:1011CA00FBFF013600F6FFFCFF013900F5FFFDFFCA
:1011DA00013900F5FFFDFF013D00F4FFFEFF01416B
:1011EA0000F3FFFFFF014600F2FFFFFF013200F6A6
:1011FA00FF010001C60200008E00015B00EEFFFE47
:10120A00FF015100F0FFFDFF014800F3FFFAFF0163
:10121A004100F5FFF9FF013C00F7FFF8FF013A0032
:10122A00FAFFF6FF013600FCFFF6FF013C00FFFF64
:10123A00F4FF0128000100F8FF0129000200F8FF6D
:10124A000126000300F9FF012B000500F9FF012E1A
:10125A00000700FAFF012F000800FBFF0133000915
:10126A0000FBFF013F000C00FCFF01000000000032
:10127A00000201000000000001320000000000012D
:10128A00CE003F006A0002000000000000013200A8
:10129A0000000000011202000096FF0141000D004B
:1012AA000100013E000C0003000134000A000300A3
:1012BA00012F00080005000140000A000800013D56
:1012CA000007000A00011B0002000500011B0002C2
:1012DA00000500013C0001000C00013700FFFF0B74
:1012EA0000012F00FDFF0900013600FAFF09000185
:1012FA003500F9FF0800013D00F6FF0700013C0038
:10130A00F5FF0500014400F3FF0400014600F2FF67
:10131A0001000100000000000002010000000000BE
:10132A000132000000000001900164FF4AFF020040
:10133A0000000000000132000000000001A200FBD2
:10134A00FFE0FF012D00F7FFFFFF012600F9FFFD77
:10135A00FF011D00FBFFFDFF012000FBFFFCFF0159
:10136A002700FBFFFAFF012B00FDFFF8FF012E000B
:10137A00FEFFF7FF013200FFFFF6FF013200010016
:10138A00F6FF0133000200F6FF012B000300F8FF0D
:10139A000127000500FAFF012A000600FAFF012BC7
:1013AA00000700FBFF012B000800FDFF012F0009C9
:1013BA0000FDFF0160001300FEFF019B001F0000FB
:1013CA0000012B00F9FF0500012A00FAFF060001BF
:1013DA002700FBFF0600012800FCFF07000124008C
:1013EA00FCFF0600012400FEFF0700012800FFFFA2
:1013FA000800012800FFFF0800012D000100090074
:10140A00012D0001000900012F0003000900012D30
:10141A00000400080001280004000700012E00064D
:10142A00000700012E00070006000132000800062E
:10143A000001330009000500013100090004000120
:10144A0036000A0004000134000A000300016B00A0
:10145A00150004000173001700010001500010007C
:10146A0000000151001000FEFF0148000E00FDFFC0
:10147A00014A000E00FBFF014A000E00FBFF01417A
:10148A00000B00F9FF0140000A00F8FF01390008CB
:10149A0000F8FF013D000700F6FF013C000500F5DA
:1014AA00FF0138000200F5FF0141000100F3FF01CE
:1014BA0028000000F8FF012900FEFFF8FF012400C0
:1014CA00FEFFF9FF012800FCFFF9FF012800FCFFDD
:1014DA00F9FF012E00FAFFF9FF012E00F9FFFAFFCA
:1014EA00012B00F9FFFBFF0187001B00000001969A
:1014FA00000000E2FF01DE033AFF0000017D00E781
:10150A00FF0000016900EBFF0200015600EFFF0334
:10151A0000014400F3FF0400013800F6FF05000152
:10152A003D00F6FF0700013500F8FF0700013D0006
:10153A00F9FF0A00013A00FAFF0A00013F00FCFF26
:10154A000C00013D00FEFF0C00014600FFFF0E00EB
:10155A0001500001001000014E0004000F00014874
:10156A000006000D0001440008000B0001200004E1
:10157A0000050001270006000500012200060003FD
:10158A0000012600070003000124000700020001F1
:10159A0029000800020001550011000100010000A5
:1015AA0000000000020100000000000132000000FB
:1015BA00000001EA008A00E5FF02000000000000C6
:1015CA0001320000000000016900EBFFFFFF015B30
:1015DA0000EEFFFDFF014F00F1FFFBFF012200FAC1
:1015EA00FFFDFF012200FAFFFDFF013C00F7FFF8B3
:1015FA00FF013900F9FFF7FF013400FDFFF6FF0193
:10160A003300FEFFF6FF0138000200F5FF01340047
:10161A000300F6FF0139000700F7FF013C0009004B
:10162A00F8FF011D000500FDFF0126000700FDFF70
:10163A00014A000E00FBFF015B001200FDFF01647E
:10164A00001400FFFF01640014000100015600119C
:10165A00000300014F000F0005000145000C0007C0
:10166A0000013C00090008000139000700090001D7
:10167A0031000400090001370001000B00013200AB
:10168A00FFFF0A00013600FCFF0A00013900F9FFDA
:10169A000900013C00F7FF0800014300F4FF0600BF
:1016AA00014A00F2FF0500015600EFFF0300015F47
:1016BA0000EDFF010001000000000000020100002F
:1016CA000000000132000000000001770176FF4EA1
:1016DA00FF020000000000000132000000000001CB
:1016EA00A200FBFFE0FF012D00F7FFFFFF0126002C
:1016FA00F9FFFDFF011D00FBFFFDFF012000FBFFBD
:10170A00FCFF012700FBFFFAFF012B00FDFFF8FF9A
:10171A00012E00FEFFF7FF013200FFFFF6FF013244
:10172A00000100F6FF0133000200F6FF012B00035F
:10173A0000F8FF0127000500FAFF012A000600FA57
:10174A00FF012B000700FBFF012B000800FDFF0132
:10175A002F000900FDFF0160001300FEFF019B003E
:10176A001F000000012B00F9FF0500012A00FAFF03
:10177A000600012700FBFF0600012400FCFF06000B
:10178A00012800FCFF0700012400FEFF07000128D2
:10179A0000FFFF0800012800FFFF0800012D0001DB
:1017AA00000900012D0001000900012F00030009B2
:1017BA000001280004000700012D000400080001B0
:1017CA002E0006000700012E000700060001320065
:1017DA000800060001330009000500013100090074
:1017EA0004000136000A0004000134000A00030064
:1017FA00016B00150004000173001700010001507D
:10180A00001000FFFF0150001000FFFF0148000E0A
:10181A0000FDFF014A000E00FBFF014A000E00FB1B
:10182A00FF0141000B00F9FF0140000A00F8FF0127
:10183A0039000800F8FF013D000700F6FF013C00EF
:10184A000500F5FF0138000200F5FF014100010023
:10185A00F3FF0128000000F8FF012900FEFFF8FF4E
:10186A00012400FEFFF9FF012800FCFFF9FF01280F
:10187A0000FCFFF9FF012E00FAFFF9FF012E00F923
:10188A00FFFAFF012B00F9FFFBFF0187001B000095
:10189A00000196000000E2FF01DE033AFF000001AA
:1018AA007D00E7FF0000016900EBFF02000156001E
:1018BA00EFFF0300014400F3FF0400013800F6FFC4
:1018CA000500013D00F6FF0700013500F8FF07009B
:1018DA00013D00F9FF0A00013A00FAFF0A00013F40
:1018EA0000FCFF0C00013D00FEFF0C00014600FF5A
:1018FA00FF0E0001500001001000014E0004000F0D
:10190A000001480006000D0001440008000B000118
:10191A002000040005000124000600040001240040
:10192A000600040001260007000300012400070046
:10193A0002000129000800020001550011000100FF
:10194A000100000000000002010000000000013256
:10195A00000000000001EA008A00E5FF0200000022
:10196A0000000001320000000000016900EBFFFFE7
:10197A00FF015B00EEFFFDFF014F00F1FFFBFF01DE
:10198A002200FAFFFDFF012200FAFFFDFF013C00E1
:10199A00F7FFF8FF013900F9FFF7FF013400FDFFF7
:1019AA00F6FF013800FEFFF5FF0133000200F6FFE3
:1019BA000134000300F6FF0139000700F7FF013C7C
:1019CA00000900F8FF011D000500FDFF01280007BE
:1019DA0000FCFF0149000E00FCFF015B001200FD44
:1019EA00FF0164001400FFFF0164001400010001FC
:1019FA00560011000300014F000F000500014500C9
:101A0A000C000700013C000900080001390007002A
:101A1A0009000131000400090001370001000B0030
:101A2A00013200FFFF0A00013600FCFF0A000139FB
:101A3A0000F9FF0900013C00F7FF0800014300F428
:101A4A00FF0600014A00F2FF0500015600EFFF03FE
:101A5A0000015F00EDFF010001000000000000022C
:101A6A0001000000000001320000000000018D01A9
:101A7A0089FF32FF0200000000000001320000006E
:101A8A00000001960000001E00012C063C01000027
:101A9A0001A5000000DFFF01300290FF0000012BCA
:101AAA00000700FBFF012A000600FAFF01270005D4
:101ABA0000FAFF0127000500FAFF0126000300F9DA
:101ACA00FF0124000200F9FF0124000200F9FF01CE
:101ADA0028000000F8FF012D000000F7FF0129008F
:101AEA00FEFFF8FF012900FEFFF8FF012D00FCFFB1
:101AFA00F8FF012F00FBFFF8FF012B00FBFFF9FFA6
:101B0A00012E00F9FFFAFF012B00F9FFFBFF012F5D
:101B1A0000F8FFFBFF013100F7FFFCFF013600F67A
:101B2A00FFFCFF013400F6FFFDFF013900F5FFFD60
:101B3A00FF013C00F4FFFFFF017800E8FFFEFF0110
:101B4A004600F2FF0000014700F2FF0200013D00DB
:101B5A00F4FF0200013D00F4FF0200013B00F5FF23
:101B6A000400013600F6FF0400013300F7FF050008
:101B7A00013300F7FF0500013100F9FF0700012ECC
:101B8A0000F9FF0600012B00FBFF0700012B00FBF9
:101B9A00FF0700012D00FCFF0800012400FEFF07DB
:101BAA0000012900FEFF0800012D000000090001C4
:101BBA002800000008000129000200080001260090
:101BCA0003000700012600030007000127000500A3
:101BDA000600012A0006000600012E000700060082
:101BEA00012F0008000500019100E3FF0000020137
:101BFA0000000000000132000000000001C1007472
:101C0A000000000200000000000001320000000095
:101C1A0000015F00EDFFFFFF015000F0FFFFFF0131
:101C2A004800F2FFFDFF013600F6FFFCFF01280025
:101C3A00F9FFFCFF012700FAFFFBFF012000FBFF71
:101C4A00FCFF012300FBFFFBFF012200FDFFFAFF5F
:101C5A00011B00FEFFFBFF012000FEFFFAFF01232C
:101C6A00000000F9FF0132000100F6FF0131000413
:101C7A0000F7FF0139000700F7FF0140000A00F8EA
:101C8A00FF0145000C00F9FF0154001000FBFF01A1
:101C9A0056001100FDFF0169001500FFFF016900F0
:101CAA0015000100015B0012000300014F000F0044
:101CBA0005000122000600030001220006000300BD
:101CCA00013C000900080001350007000800013640
:101CDA000004000A0001320001000A00013200FF7C
:101CEA00FF0A00013600FCFF0A00013900F9FF096A
:101CFA0000014000F6FF0800014300F4FF0600015E
:101D0A004F00F1FF0500015600EFFF0300016400D8
:101D1A00ECFF0100010000000000000201000000C9
:101D2A00000001320000000000011001FFFF5DFF0A
:101D3A000200000000000001320000000000014B18
:101D4A00000F00FFFF0146000E00FFFF0148000ED2
:101D5A0000FDFF013E000C00FDFF013B000B00FCF3
:101D6A00FF013C000B00FBFF0136000900FAFF01EE
:101D7A0035000800F9FF012A000600FAFF012B00CE
:101D8A000500F9FF0128000400F9FF0128000400FA
:101D9A00F9FF012B000300F8FF0129000200F8FFF8
:101DAA000128000100F8FF012D000000F7FF0132B1
:101DBA00000000F6FF012E00FEFFF7FF012E00FED5
:101DCA00FFF7FF012B00FDFFF8FF012F00FBFFF8D3
:101DDA00FF012B00FBFFF9FF012E00FAFFF9FF01BB
:101DEA003200F8FFFAFF013200F8FFFAFF012F0074
:101DFA00F8FFFBFF013800F6FFFBFF013400F6FF96
:101E0A00FDFF013900F5FFFDFF013D00F4FFFEFF74
:101E1A00014100F3FFFFFF014100F3FF00000169E8
:101E2A0000EBFF0000016000EDFF0200015200F02C
:101E3A00FF0400014A00F2FF0500014300F4FF0617
:101E4A0000013D00F6FF0700014000F7FF0900010D
:101E5A004000F8FF0A00013F00FAFF0B00013C00B6
:101E6A00FBFF0B00013D00FEFF0C00013C00FFFFE1
:101E7A000C0001320000000A00012E0002000900D5
:101E8A00012E0002000900012D0004000800012DA6
:101E9A000004000800012F0005000800012E0007B9
:101EAA0000060001310007000700013200080006A1
:101EBA0000013300090005000136000A0004000190
:101ECA0034000A000300013E000C000300013D003B
:101EDA000C0002000146000E0001000146000E003F
:101EEA0001000100000000000002010000000000E3
:101EFA00013200000000000139000000DEFF02008C
:101F0A00000000000001320000000000016900EB3F
:101F1A00FFFFFF015B00EEFFFDFF014F00F1FFFB3A
:101F2A00FF012200FAFFFDFF012400FAFFFCFF0176
:101F3A004000F6FFF8FF013D00F9FFF6FF01360009
:101F4A00FCFFF6FF013C00FFFFF4FF013C0001002B
:101F5A00F4FF0136000400F6FF013D000700F6FF1A
:101F6A000140000A00F8FF0124000600FCFF0122DC
:101F7A00000600FDFF0154001000FBFF015B001288
:101F8A0000FDFF0169001500FFFF01640014000154
:101F9A000001560011000300014F000F0005000167
:101FAA002600070003000120000500040001430089
:101FBA000A00090001390007000900013B0004007A
:101FCA000B0001370001000B00013C00FFFF0C0071
:101FDA00013600FCFF0A00013D00F9FF0A0001403A
:101FEA0000F6FF0800012000FBFF0400012600F9AB
:101FFA00FF0300014F00F1FF0500015B00EEFF0344
:10200A0000016400ECFF0100010000000000000272
:10201A000100000000000132000000000001BC01C4
:10202A00B0FF02FF020000000000000132000000C1
:10203A00000001AC00DEFFFBFF014300FDFF0D00C5
:10204A00013C00FFFF0C00012800010008000123E9
:10205A00000100070001240002000700011D00031F
:10206A000005000119000300040001200005000416
:10207A000001190004000300011D0005000300010E
:10208A002300070001000133000A00020001910049
:10209A001D00010001940284000000017300000089
:1020AA0017000196001E0000000173000000E9FFFE
:1020BA00011D013900000001C9001700DFFF01906E
:1020CA0001B0FF000001A0000000E0FF019600E25D
:1020DA00FF000001A00000002000019E027AFF001C
:1020EA0000014600F2FF0000012300F9FFFFFF0193
:1020FA001D00FBFFFDFF011500FDFFFDFF011B0099
:10210A00FEFFFBFF011E00FFFFFAFF01470002006E
:10211A00F2FF0100000000000002010000000000C0
:10212A00013200000000000158075AFF5C04020057
:10213A0000000000000132000000000001C701A8F1
:10214A00FFE9FF0141000000F3FF015C014400F1D7
:10215A00FF014C00F1FFFEFF011001CBFFF4FF016C
:10216A0041000000F3FF01C7015800E9FF013C00EC
:10217A0000000C00010701CDFF0D00015700EFFF21
:10218A0004000157001100040001050133000B008F
:10219A00013C0000000C00010601CDFF0C000161AA
:1021AA0000EDFF0400016100130004000106013381
:1021BA00000C0001410000000D00010000000000B9
:1021CA0000020100000000000132000000000001CE
:1021DA00FF00A8FF83FF0200000000000001320098
:1021EA000000000001C6015800160001410000006D
:1021FA00F3FF010501CDFFF5FF016200EDFFFBFFD3
:10220A000161001300FCFF0105013300F5FF0141E4
:10221A00000000F3FF010501CDFFF5FF015700EFB4
:10222A00FFFCFF0157001100FCFF0107013300F317
:10223A00FF013C000000F4FF01C701A8FF170001DD
:10224A00410000000D0001100135000C00014C0096
:10225A000F000300015C01BCFF0F000141000000F8
:10226A000D00020100000000000132000000000021
:10227A0001AC00000099FF020000000000000132DA
:10228A00000000000001C60158001600013C0000D1
:10229A0000F4FF010601CDFFF4FF016200EDFFFB30
:1022AA00FF0160001300FDFF0106013300F4FF0186
:1022BA0041000000F3FF010501CDFFF5FF015700C2
:1022CA00EFFFFCFF0157001100FCFF01070133007B
:1022DA00F3FF013C000000F4FF01C701A8FF17004B
:1022EA0001410000000D0001100135000C00014CF5
:1022FA00000F000300015C01BCFF0F000141000058
:10230A00000D000201000000000001320000000080
:10231A0000019B000000A3FF020000000000000172
:10232A0032000000000001550011000000014600C3
:10233A000000F2FF015500EFFF0000014600000017
:10234A000E0002010000000000013200000000003F
:10235A000197001C00AAFF020000000000000132E1
:10236A000000000000014100FFFFF3FF012400F913
:10237A00FF0200012000FAFF0200011900FCFF031E
:10238A0000012000FBFF0400011D00FDFF05000104
:10239A001B00FEFF0500011B00FEFF0500011E00D9
:1023AA0000000600012800010008000124000200C4
:1023BA0007000124000400060001230005000500AF
:1023CA0001240006000400012B0008000300012E6E
:1023DA0000090002000132000A0000000137000B68
:1023EA00000000012E000900FEFF012B000800FD7D
:1023FA00FF0128000700FCFF0123000500FBFF0185
:10240A0024000400FAFF0126000300F9FF0123005B
:10241A000000F9FF0123000000F9FF012200FDFF7F
:10242A00FAFF012200FDFFFAFF012700FAFFFBFF76
:10243A00012400FAFFFCFF012B00F8FFFDFF012E2B
:10244A0000F7FFFEFF013700F5FFFFFF011500FC53
:10245A00FF010001130100003700012300F9FFFF0B
:10246A00FF012000FAFFFEFF011B00FBFFFEFF0138
:10247A001600FCFFFEFF011900FDFFFCFF0115001D
:10248A00FDFFFDFF011500FFFFFCFF011900FFFF23
:10249A00FBFF011E000100FAFF0120000400FBFF00
:1024AA000123000500FBFF012B000800FDFF0100CE
:1024BA0000000000000201000000000001320000DC
:1024CA00000000015000190029000200000000006D
:1024DA00000132000000000001CD000000D7FF011A
:1024EA002D000900010001260007000300011C005D
:1024FA000400040001150003000300011600020095
:10250A000400011900000005000114000000040085
:10251A00011600FEFF0400011200FEFF0300011570
:10252A0000FDFF0300011900FCFF0300011600FC77
:10253A00FF0200011900FBFF0100011900FBFF0166
:10254A00000100000000000002010000000000017C
:10255A00320000000000019700C4FFBCFF02000027
:10256A000000000001320000000000013E00FDFFF3
:10257A00F4FF011900FBFFFFFF011900FCFFFDFF3B
:10258A00011D00FDFFFBFF012900FEFFF8FF0124EA
:10259A00000200F9FF0122000300FAFF01200005F2
:1025AA0000FCFF0120000600FEFF0123000700FFD8
:1025BA00FF0141000D000000012400FAFF040001A0
:1025CA001D00FDFF0500011B00FEFF0500011E00A6
:1025DA00FFFF06000123000100070001240002009A
:1025EA00070001200004000500012700060005007D
:1025FA0001260007000300012B0008000300012840
:10260A000008000100012D0009000100013C000C36
:10261A0000FFFF0139000B00FDFF0138000A00FB33
:10262A00FF012E000700FAFF0116000200FCFF015D
:10263A0016000200FCFF0115000100FCFF01190051
:10264A000000FBFF011E000000FAFF012200FDFF4F
:10265A00FAFF012000FCFFFBFF012300FBFFFBFF49
:10266A000132000A0000000137000000F5FF017C7A
:10267A0001B4FF0000015A00EEFF0100011E00FA3A
:10268A00FF0100011900FBFF0100012F00F8FF05FF
:10269A0000012E00FAFF0700012D00FCFF080001CF
:1026AA003200FFFF0A0001230001000700011900A0
:1026BA0001000500011B0002000500011D000300C6
:1026CA00050001190004000300011D0005000300B4
:1026DA00011E00060001000123000700000001009E
:1026EA0000000000000201000000000001320000AA
:1026FA00000000015A003500F6FF02000000000049
:10270A000001320000000000012800F8FF0000016B
:10271A002300F9FFFFFF012000FAFFFEFF011D0061
:10272A00FBFFFDFF011500FDFFFDFF011500FDFF89
:10273A00FDFF011500FFFFFCFF011500FFFFFCFF75
:10274A000115000100FCFF0115000100FCFF011545
:10275A00000300FDFF0119000300FCFF011B000537
:10276A0000FEFF0120000600FEFF011E000600FF1A
:10277A00FF012800080000000128000800000001ED
:10278A001E000600010001200006000200011D00D3
:10279A0005000300011500030003000115000300F2
:1027AA0003000115000100040001150001000400E6
:1027BA00011500FFFF0400011500FFFF04000115C9
:1027CA0000FDFF0300011500FDFF0300011D00FBD2
:1027DA00FF0300011B00FBFF0200012300F9FF01B8
:1027EA0000012300F9FF00000100000000000002C0
:1027FA000100000000000132000000000001910009
:10280A00CBFFBBFF02000000000000013200000005
:10281A000000013E00FDFFF4FF011900FBFFFFFF6E
:10282A00011900FCFFFDFF012200FDFFFAFF012450
:10283A0000FEFFF9FF0129000200F8FF011D000355
:10284A0000FBFF0120000500FCFF0122000600FD3D
:10285A00FF012300070000000141000D00FFFF01F6
:10286A002700FAFF0500011D00FDFF0500011B00FE
:10287A00FEFF0500011E00FFFF0600012300010004
:10288A0007000120000200060001240004000600DF
:10289A000124000600040001280007000400012B9F
:1028AA00000800030001280008000100012D0009AA
:1028BA00000100013C000C00FFFF0139000B00FD84
:1028CA00FF0138000A00FBFF012E000700FAFF0192
:1028DA0016000200FCFF0116000200FCFF011500B1
:1028EA000100FCFF0119000000FBFF011E000000AF
:1028FA00FAFF012200FDFFFAFF012000FCFFFBFFA7
:10290A00012300FBFFFBFF0132000A000000013730
:10291A00000000F5FF017C01B4FF0000015A00EE3F
:10292A00FF0100011E00FAFF0100011900FBFF016F
:10293A0000012F00F8FF0500012A00FAFF06000136
:10294A003100FCFF0900013200FFFF0A00011E00EE
:10295A0001000600011E0001000600011B00020022
:10296A00050001190003000400011C000400040012
:10297A00011B0005000200012000060002000123DD
:10298A000007000000010000000000000201000032
:10299A0000000001320000000000015A003500F674
:1029AA00FF020000000000000132000000000001E8
:1029BA002800F8FF0000012400F9FFFEFF011E00B5
:1029CA00FAFFFFFF011D00FBFFFDFF011500FDFFE0
:1029DA00FDFF011500FDFFFDFF011500FFFFFCFFD4
:1029EA00011500FFFFFCFF0115000100FCFF0115A6
:1029FA00000100FCFF0119000300FCFF01150003A0
:102A0A0000FDFF011B000500FEFF0120000600FE7D
:102A1A00FF011E000600FFFF0128000800FFFF015A
:102A2A00280008000100011E000600010001200024
:102A3A0006000200011B0005000200011900030044
:102A4A000400011500030003000115000100040041
:102A5A0001150001000400011500FFFF0400011523
:102A6A0000FFFF0400011500FDFF0300011500FD32
:102A7A00FF0300011D00FBFF0300011900FBFF011A
:102A8A0000012400F9FF0200012300F9FF00000100
:102A9A0000000000000002010000000000013200F6
:102AAA0000000000016F00F7FFBEFF0200000000F7
:102ABA00000001320000000000014B000F0000007E
:102ACA0001C3000000D9FF014B00F1FF000001C360
:102ADA00000000270002010000000000013200008F
:102AEA00000000017B00DBFFC0FF020000000000C5
:102AFA00000132000000000001370000000B000155
:102B0A0062027A000000013C000000F4FF01DC00D0
:102B1A00D4FF00000124000600FCFF011D00030091
:102B2A00FBFF011D000300FBFF011E000000FAFF6E
:102B3A000123000000F9FF012200FDFFFAFF012432
:102B4A0000FCFFFAFF012000FBFFFCFF012800F94F
:102B5A00FFFCFF012900F8FFFEFF012900F8FFFE34
:102B6A00FF012D00F7FFFFFF013700F5FF0100010C
:102B7A003300F6FF0200012B00F8FF0300012800D2
:102B8A00F9FF0400012300FBFF0500012000FCFF00
:102B9A000500012000FEFF0600011E00FFFF0600DF
:102BAA00011E0001000600012000020006000120AB
:102BBA00000400050001240006000400013700F5A6
:102BCA00FF000002010000000000013200000000C6
:102BDA0000014B002D00000002000000000000016F
:102BEA00320000000000014600F2FFFFFF012F0043
:102BFA00F7FFFDFF011D00FBFFFDFF011C00FCFFAD
:102C0A00FCFF011600FEFFFCFF011900FFFFFBFF9E
:102C1A000115000100FCFF0110000100FDFF011970
:102C2A00000300FCFF0119000400FDFF011B000561
:102C3A0000FEFF011B000500FEFF0123000700FF45
:102C4A00FF0128000800FFFF012800080001000119
:102C5A00230007000100011E0006000100011D00FB
:102C6A00050003000115000300030001150003001D
:102C7A000300011600020004000114000000040011
:102C8A0001140000000400011200FEFF03000119F4
:102C9A0000FDFF0400011500FDFF0300011D00FBFC
:102CAA00FF0300011E00FAFF0100012400F9FF02E0
:102CBA0000012300F9FF00000100000000000002EB
:102CCA00010000000000013200000000000169005C
:102CDA00FFFFC1FF020000000000000132000000F7
:102CEA000000013C000C00FFFF0133000A00FEFF58
:102CFA00012D000800FCFF012B000700FBFF01204B
:102D0A00000400FBFF011D000300FBFF012000027D
:102D1A0000FAFF0123000000F9FF0123000000F977
:102D2A00FF012600FDFFF9FF011D00FDFFFBFF016A
:102D3A002A00FAFFFAFF012400FAFFFCFF012B0028
:102D4A00F8FFFDFF012E00F7FFFEFF013200F6FF3C
:102D5A000000014B00F1FF0100011E00FAFF010013
:102D6A00011B00FBFF0200013300F7FF05000131E0
:102D7A0000F9FF0700013100FCFF0900012D00FFE7
:102D8A00FF090001280001000800012000020006D6
:102D9A0000012400040006000123000500050001CB
:102DAA00240006000400012B000800030001330080
:102DBA000A0002000132000A0001000100000000BE
:102DCA0000000201000000000001320000000000C3
:102DDA000116000000F3FF020000000000000132AB
:102DEA000000000000012800F8FF0000012400F99B
:102DFA00FFFEFF011E00FAFFFFFF011900FCFFFDA5
:102E0A00FF011900FCFFFDFF011900FDFFFCFF0196
:102E1A001500FFFFFCFF011900FFFFFBFF01150072
:102E2A000100FCFF0115000100FCFF01190003006D
:102E3A00FCFF0119000400FDFF011D000500FDFF54
:102E4A00011B000500FEFF0128000800FFFF012802
:102E5A00000800000001230007000000012300070A
:102E6A0000010001200006000200011D0005000308
:102E7A00000115000300030001190003000400010A
:102E8A0015000100040001150001000400011900E9
:102E9A00FFFF0500011500FFFF0400011900FDFFF7
:102EAA000400011500FDFF0300011D00FBFF0300E4
:102EBA00011E00FAFF0100012400F9FF02000128A7
:102ECA0000F8FF00000100000000000002010000FD
:102EDA000000000132000000000001AB00E1FF9E8B
:102EEA00FF020000000000000132000000000001A3
:102EFA004200F3FFFEFF012D00FFFF0900011E0043
:102F0A0000000600011B0002000500011500030075
:102F1A00030001160004000200012300070001005B
:102F2A000137000B00010001FF0033000000012DF2
:102F3A0000000009000137000B000000012D00000D
:102F4A0000F7FF016E0016000000014F000900F3B0
:102F5A00FF019B00E1FF0000013C000000F4FF01BB
:102F6A003700F5FF0000013C0000000C00010401DD
:102F7A00CCFF0000012800F8FF0000011500FDFF4A
:102F8A00FDFF011500FFFFFCFF0119000000FBFF18
:102F9A0001000000000000020100000000000132F0
:102FAA000000000000012200F3FFF0FF0200000011
:102FBA00000000013200000000000155001100006D
:102FCA00000146000000F2FF015500EFFF0000017A
:102FDA00460000000E00020100000000000132005D
:102FEA00000000000196002000ACFF020000000073
:102FFA00000001320000000000013D00FEFFF4FF66
:10300A00012300F9FF0100012000FAFF020001225A
:10301A0000FAFF0300011C00FCFF0400011C00FC75
:10302A00FF0400011D00FDFF0500012000FEFF0650
:10303A000001190000000500012800010008000134
:10304A0020000200060001240004000600012300FB
:10305A000500050001240006000400012B000800F9
:10306A000300012D00090001000137000B000100D7
:10307A000141000D00FFFF013E000C00FDFF011B96
:10308A00000500FEFF0119000400FDFF01190004FC
:10309A0000FDFF0119000300FCFF012D000400F8E8
:1030AA00FF0132000100F6FF0119000000FBFF01D9
:1030BA001E00FFFFFAFF011900FDFFFCFF011900C6
:1030CA00FDFFFCFF011C00FCFFFCFF011D00FBFFD4
:1030DA00FDFF011B00FBFFFEFF012300F9FFFFFFBD
:1030EA00013D00FEFF0C0001290008000200012436
:1030FA000006000400011D0003000500011E000176
:10310A0000060001140000000400011600FEFF047E
:10311A0000011900FDFF0400011500FDFF03000175
:10312A001D00FBFF0300012000FAFF02000123003B
:10313A00F9FF0100012800F8FF0000012800F8FF4C
:10314A000000012300F9FFFFFF012000FAFFFEFF44
:10315A00011D00FBFFFDFF011500FDFFFDFF01152D
:10316A0000FDFFFDFF011500FFFFFCFF011500FF39
:10317A00FFFCFF0124000200F9FF0124000400FA09
:10318A00FF0112000300FEFF0116000400FEFF010A
:10319A002E000900FEFF01000000000000020100ED
:1031AA0000000000013200000000000124000C00B1
:1031BA00EEFF0200000000000001320000000000E3
:1031CA00013C000C00FFFF0133000A00FEFF012D45
:1031DA00000800FCFF012B000700FBFF0120000490
:1031EA0000FBFF011D000300FBFF0120000200FAA3
:1031FA00FF0123000000F9FF0123000000F9FF018D
:10320A002600FDFFF9FF012200FDFFFAFF0127005A
:10321A00FAFFFBFF012400FAFFFCFF012B00F8FF75
:10322A00FDFF012E00F7FFFEFF013200F6FF00004E
:10323A00014B00F1FF0100011E00FAFF0100011B12
:10324A0000FBFF0200013300F7FF0500013100F91E
:10325A00FF0700013100FCFF0900012D00FFFF09F3
:10326A0000012300010007000124000200070001F9
:10327A0024000400060001230005000500012400C3
:10328A0006000400012B00080003000133000A00B5
:10329A0002000132000A00010001000000000000E3
:1032AA0002010000000000013200000000000116C7
:1032BA00000000F3FF0200000000000001320000DD
:1032CA00000000012800F8FFFFFF012300F9FFFFBB
:1032DA00FF012000FAFFFEFF011600FCFFFEFF01BE
:1032EA001C00FCFFFCFF011500FDFFFDFF0115009E
:1032FA00FFFFFCFF011900FFFFFBFF0115000100A2
:10330A00FCFF0115000100FCFF0119000300FCFF8E
:10331A000119000400FDFF011D000500FDFF011B4E
:10332A00000500FEFF0128000800FFFF0128000831
:10333A0000FFFF012300070001000123000700012D
:10334A000001200006000200011D00050003000123
:10335A001500030003000119000300040001150011
:10336A000100040001150001000400011900FFFF1B
:10337A000500011500FFFF0400011500FDFF030011
:10338A00011900FDFF0400011B00FBFF02000120E0
:10339A0000FAFF0200012300F9FF0100012800F8EA
:1033AA00FF0100010000000000000201000000000F
:1033BA000001320000000000018B00D4FFB9FF02B7
:1033CA000000000000000132000000000001B80106
:1033DA00580000000137000000F5FF013C00F4FF2F
:1033EA0000000124000600FCFF0124000400FAFF8B
:1033FA000122000300FAFF0123000100F9FF012363
:10340A0000FFFFF9FF012200FDFFFAFF012300FB85
:10341A00FFFBFF012000FAFFFEFF012B000700FB64
:10342A00FF0127000500FAFF0120000200FAFF0150
:10343A001E000100FAFF0119000000FBFF0119003C
:10344A00FFFFFBFF011900FDFFFCFF011500FDFF57
:10345A00FDFF011900FCFFFDFF011B00FBFFFEFF42
:10346A00011E00FAFFFFFF012300F9FF00000131EE
:10347A0001C3FF0000013C0000000C0001180138E4
:10348A0000000001230007000100011E00060001E0
:10349A0000011000030001000115000300030001F0
:1034AA0016000200040001140000000400010F00CD
:1034BA0000000300011500FFFF0400011200FEFFD7
:1034CA000300011200FDFF0200011500FDFF0300C9
:1034DA00011900FBFF0100013D00F4FF020001FF9A
:1034EA0000CDFF0000013C0000000C00011D013965
:1034FA00000000012D000900010001200006000261
:10350A000001120003000200010B00010002000189
:10351A001E000100060001190000000500011D003F
:10352A00FDFF0500011C00FCFF0400012000FAFF5A
:10353A000200012900F8FF0200013200F6FF000034
:10354A0001E600D2FF000001410000000D00020167
:10355A0000000000000132000000000001ED05CB70
:10356A000089FC0200000000000001320000000097
:10357A000001A400F5FFE1FF01A100F7FFE1FF014F
:10358A002201F1FFC8FF010501F5FFCDFF01DA00B5
:10359A00F9FFD5FF01B100FBFFDDFF018700FEFF48
:1035AA00E5FF016E00FEFFEAFF02010000000000D5
:1035BA000132000000000001F8013E00280102006B
:1035CA0000000000000132000000000001800280BB
:1035DA00FF000002010000000000013200000000AC
:1035EA0000010C02EC0030FF0200000000000001A4
:1035FA0032000000000001AB00F7FF210001950036
:10360A00F6FF1C00019600F5FF1C00019D00F4FF67
:10361A001D0001C000F0FF230001CE00ECFF2400D2
:10362A00016300F6FF1100016100F5FF100001645B
:10363A0000F4FF1000016000F4FF0F00012A00FAF5
:10364A00FF0600012700FAFF0500012400FAFF0423
:10365A0000012000FAFF0200012000FAFF02000127
:10366A001E00FAFF0000013C00F4FF0000013D00CB
:10367A00F4FFFEFF014200F3FFFEFF014200F3FFE9
:10368A00FEFF014600F2FF0000013700F5FF0000CF
:10369A00012D00F7FFFFFF012B00F8FFFDFF0120BE
:1036AA0000FBFFFCFF010E00FEFFFEFF010F000002
:1036BA0000FDFF011000FFFFFDFF0115000100FCE6
:1036CA00FF012D000400F8FF0140000800F6FF0189
:1036DA0020000400FBFF0124000200F9FF012E0074
:1036EA000200F7FF012D000000F7FF012D00FFFF88
:1036FA00F7FF012E00FEFFF7FF012800FCFFF9FF8C
:10370A00012700FBFFFAFF0201000000000001325E
:10371A000000000000019E02FF00C9FE0200000036
:10372A0000000001320000000000011E0006000037
:10373A00000115000400010001120003000200014B
:10374A00160002000400011B000200050001190016
:10375A0001000500014600FFFF0E00014C00FEFFBC
:10376A000F00014C00FDFF0F00018E00FBFF1C0043
:10377A00018F00FAFF1C0002010000000000013264
:10378A000000000000012902E9FEB4000200000066
:10379A0000000001320000000000015D00EEFFFBA6
:1037AA00FF014700F2FFFEFF013700F5FF000001AD
:1037BA002F00F7FF0300012700FAFF050001270089
:1037CA00FBFF0600012600FDFF0700012E00FEFF99
:1037DA000900015600FDFF1100012D00FFFF09003D
:1037EA00012900FEFF0800012600FDFF0700012055
:1037FA0000FCFF0500012400FAFF0400012800F87C
:10380A00FF0100018A01EFFFB3FF011E000000FA69
:10381A00FF0119000100FBFF0136000400F6FF0159
:10382A003A000600F6FF0136000600F7FF016000C5
:10383A000C00F1FF0128000400F9FF01200002003A
:10384A00FAFF010B00FFFFFEFF011000FFFFFDFF63
:10385A00012E00F9FFFAFF018A00EBFFEEFF014B90
:10386A0000F4FFF7FF014A00F6FFF5FF014300F7F6
:10387A00FFF6FF011D00FDFFFBFF011B00FEFFFB22
:10388A00FF014B01F3FFBFFF010401F6FFCDFF016A
:10389A0019000500000001190005000100011600C9
:1038AA0004000200011600040002000135000700AE
:1038BA000800013A0006000A000194000C001B00EF
:1038CA00015E000800110001600009001100011DDD
:1038DA000003000500011C00040004000144000B61
:1038EA00000800014A000D000700014A000E000509
:1038FA00000147000E00020001230007000000013A
:10390A0023000700FFFF0120000600FEFF011D0043
:10391A000500FDFF0120000500FCFF012400040052
:10392A00FAFF0131000400F7FF013E000300F4FF33
:10393A000141000100F3FF0146000000F2FF02010D
:10394A00000000000001320000000000010A000629
:10395A000000000200000000000001320000000028
:10396A000001660014000400015100100002000169
:10397A003C000C0000000133000A00FEFF012D008C
:10398A000800FCFF0132000800FAFF0135000800B8
:10399A00F9FF0143000900F6FF014E000A00F4FF97
:1039AA00014E000A00F4FF019E001200E6FF0138F2
:1039BA00012100CBFF0155000800F1FF015C00095D
:1039CA0000F0FF01BE000F00DDFF01BF000D00DCAB
:1039DA00FF01B1000A00DEFF01F7000C00D0FF0171
:1039EA00F5000A00D0FF015A000100EEFF011E0097
:1039FA00FFFFFAFF011500FFFFFCFF011200FEFFA7
:103A0A00FDFF011200FDFFFEFF011000FDFFFFFF99
:103A1A00011000FDFF0100012E00F7FF0200012F37
:103A2A0000F7FF0300013900F5FF0300013200F639
:103A3A00FF0100013200F6FF0000012E00F7FF022D
:103A4A0000013100F7FF0400013600F7FF0600010C
:103A5A003900F7FF0700013C00F8FF0900014300A5
:103A6A00F7FF0A00014400F8FF0B00018900F1FF8B
:103A7A001700019200F1FF1900018B00F2FF1800F4
:103A8A00018000F3FF16000201000000000001326D
:103A9A000000000000019B01C4FFEF0002000000CB
:103AAA0000000001320000000000015F00EDFF008D
:103ABA0000015100F0FFFEFF013D00F4FFFEFF018F
:103ACA003100F7FFFCFF011500FDFFFDFF011500A6
:103ADA00FDFFFDFF011600FEFFFCFF011500FFFFC1
:103AEA00FCFF013C00FFFFF4FF014C000200F1FF64
:103AFA000156000300EFFF0161000400EDFF0162BF
:103B0A00000500EDFF0165000700EDFF01650009F2
:103B1A0000EEFF0132000600F8FF0132000600F84D
:103B2A00FF0135000700F8FF0131000700F9FF0126
:103B3A0032000800FAFF0133000900FBFF0201000E
:103B4A000000000001320000000000011D00F1FF2A
:103B5A00090002000000000000013200000000001D
:103B6A0001FF00F6FFCEFF015601F2FFBDFF020181
:103B7A000000000000013200000000000186023D42
:103B8A0001DF000200000000000001320000000016
:103B9A0000019300F7FFE4FF018200F9FFE7FF014C
:103BAA000701F3FFCDFF019F00F9FFE1FF01C50007
:103BBA00FAFFD9FF01D400FAFFD6FF01DD00FCFFAE
:103BCA00D4FF0201000000000001320000000000E2
:103BDA00018F01F7FFEF0002000000000000013230
:103BEA000000000000017F000B00E9FF014600F21F
:103BFA00FFFFFF017D00F6FF17000141000D0001E4
:103C0A0000010000000000000201000000000001A5
:103C1A00320000000000011700F2FF00000200005D
:103C2A000000000001320000000000016A00FDFFF0
:103C3A00EBFF0172000900EBFF015D0005001200B5
:103C4A00020100000000000132000000000001270C
:103C5A0000F4FF140002000000000000013200001E
:103C6A00000000014F01BDFFFFFF0201000000003C
:103C7A000001320000000000016E004000EFFF0268
:103C8A0000000000000001320000000000010901EC
:103C9A00CBFF00000201000000000001320000001A
:103CAA000000016F003F00EBFF020000000000006F
:103CBA000132000000000001FA00CEFF00000201FC
:103CCA000000000000013200000000000179003A03
:103CDA00002C000200000000000001320000000079
:103CEA000001F2021D009400020100000000000120
:103CFA00320000000000010401D5FF6AFF02000043
:103D0A00000000000132000000000001F7021D005F
:103D1A0095000201000000000001320000000000CE
:103D2A00011D01FCFF55FF020000000000000132E6
:103D3A00000000000001BF021B008A00020100000F
:103D4A0000000001320000000000012B0002001AEE
:103D5A000002000000000000013200000000000123
:103D6A002800FFFF0800012400FEFF0700010700EA
:103D7A00FFFF0100010700FFFF0100010E00FEFF27
:103D8A00FEFF012800FCFFF9FF020100000000000D
:103D9A0001320000000000011800F2FFFEFF0200DD
:103DAA0000000000000132000000000001240002AF
:103DBA0000070001150003000300010B00020001C7
:103DCA00000141000D000000020100000000000196
:103DDA0032000000000001EF007AFF330002000009
:103DEA000000000001320000000000012600070068
:103DFA00FDFF0126000700FDFF0132000800FAFF5F
:103E0A00012E000700FAFF0135000700F8FF01360E
:103E1A00000600F7FF0136000600F7FF013A000628
:103E2A0000F6FF0138000500F6FF013B000400F52B
:103E3A00FF0139000300F5FF0133000200F6FF011C
:103E4A0037000100F5FF012D000000F7FF013200E5
:103E5A00FFFFF6FF012D00FCFFF8FF012600FDFF22
:103E6A00F9FF012300FBFFFBFF011D00FBFFFDFF24
:103E7A00012200FAFFFDFF011E00FAFFFFFF011EEB
:103E8A0000FAFFFFFF011E00FAFF0100012300F9FB
:103E9A00FF0100013F00F4FF0400014300F4FF06A4
:103EAA0000013900F7FF0700013500F8FF0700029B
:103EBA000100000000000132000000000001F300D0
:103ECA0085003C00020000000000000132000000F2
:103EDA00000001D600D7FFF4FF0201000000000035
:103EEA00013200000000000140002500F5FF020039
:103EFA0000000000000132000000000001C100DBE8
:103F0A00FF0B000201000000000001320000000067
:103F1A0000016B003F000C000200000000000001DD
:103F2A00320000000000014001400000000136019B
:103F3A003E0000000176027E00FDFF014C000F00EA
:103F4A00FEFF012D000900FFFF0110000300FFFF23
:103F5A00010B000100FEFF0110000100FDFF011925
:103F6A00000000FBFF012800FFFFF8FF010B00FF24
:103F7A00FFFEFF010B00FEFFFFFF012D00F7FFFF11
:103F8A00FF015000F0FFFFFF017B0281FF010001EA
:103F9A003B01C1FF0100014001C0FF0300010B000A
:103FAA00FEFF0100010E00FEFF0200011500FFFFE7
:103FBA0004000119000000050001190001000500B4
:103FCA0001150001000400011200020003000110A3
:103FDA0000030001000100000000000002010000CF
:103FEA00000000013200000000000147001500DB5C
:103FFA00FF02000000000000013200000000000182
:10400A00BA00EFFFDFFF015900F8FFF0FF015E0081
:10401A00F8FFEFFF0201000000000001320000007B
:10402A000000016D00EBFFC2FF020000000000006B
:10403A0001320000000000016200FBFFEDFF016099
:10404A0000FEFFEDFF016000FEFFEDFF015F00FFD4
:10405A00FFEDFF01C3000100D9FF01B9000100DB38
:10406A00FF02010000000000013200000000000110
:10407A005B014300C500020000000000000132009D
:10408A000000000001C800D8FFFFFF020100000085
:10409A00000001320000000000015002EBFE22FF86
:1040AA0002000000000000013200000000000128A8
:1040BA00000800010001260007000300012700068E
:1040CA000005000123000500050001550008000F46
:1040DA00000162000800120001B6000D0022000271
:1040EA000100000000000132000000000001F2019E
:1040FA0056001E010200000000000001320000000C
:10410A000000010C01E8FF3000020100000000007D
:10411A00013200000000000154002100DAFF020011
:10412A0000000000000132000000000001FF00EA68
:10413A00FF2E000201000000000001320000000012
:10414A0000019B00B4FFCAFF02000000000000014A
:10415A00320000000000011101E6FF3000020100F8
:10416A00000000000132000000000001EC008A009B
:10417A001F000200000000000001320000000000E1
:10418A00011C01E9FF3400020100000000000132B5
:10419A000000000000017C00E6FFBAFF02000000F8
:1041AA000000000132000000000001C201A6FF0168
:1041BA0000020100000000000132000000000001BE
:1041CA009C005C00F0FF02000000000000013200C9
:1041DA000000000001C701A5FF0200020100000063
:1041EA0000000132000000000001E60068005B00E8
:1041FA00020000000000000132000000000001BDC2
:10420A0001A7FF01000201000000000001320000C6
:10421A000000000194005900FFFF020000000000A6
:10422A000001320000000000018C01F2FFB2FF021F
:10423A0001000000000001320000000000017C00C3
:10424A0019004600020000000000000132000000D0
:10425A000000018701F2FFB3FF0201000000000025
:10426A000132000000000001CB00AAFF5600020044
:10427A00000000000001320000000000018E01F081
:10428A00FFB2FF020100000000000132000000003E
:10429A000001DD007400C0FF020000000000000100
:1042AA0032000000000001BD01A7FF010002010069
:1042BA000000000001320000000000019B004B00DA
:1042CA003700020000000000000132000000000078
:1042DA00014100F5FF070002010000000000013261
:1042EA0000000000000117000000F2FF02000000B9
:1042FA0000000001320000000000014600FFFF0E2E
:10430A00000201000000000001320000000000016C
:10431A0019000100F1FF0200000000000001320054
:10432A00000000000144000B000800020100000028
:10433A0000000132000000000001B60093FF0100F6
:10434A0002000000000000013200000000000135F8
:10435A00000700080002010000000000013200000E
:10436A00000000011B000200F0FF02000000000034
:10437A000001320000000000013900F7FF070002C7
:10438A000100000000000132000000000001F200FC
:10439A007B004D0002000000000000013200000016
:1043AA000000014400F5FF080002010000000000BF
:1043BA000132000000000001A000A0FFF9FF020086
:1043CA00000000000001320000000000018A01EF35
:1043DA00FFB3FF02010000000000013200000000EC
:1043EA0000015C001A00CFFF02000000000000017B
:1043FA00320000000000011301E7FF310002010052
:10440A000000000001320000000000016D002200DF
:10441A00C8FF020000000000000132000000000096
:10442A00013900F7FF070002010000000000013215
:10443A00000000000001A4006200F9FF0200000071
:10444A0000000001320000000000014E0007000ECB
:10445A00000201000000000001320000000000011B
:10446A00D40086FF24000200000000000001320090
:10447A000000000001410000000D000201000000E0
:10448A000000013200000000000177000800470028
:10449A0002000000000000013200000000000131AB
:1044AA0000070007000201000000000001320000BE
:1044BA000000000143026200B3FE02000000000097
:1044CA000001320000000000015101F2FFBEFF02AC
:1044DA0001000000000001320000000000016B0032
:1044EA0019003B0002000000000000013200000039
:1044FA000000014B01F3FFBFFF02010000000000B2
:10450A0001320000000000014500230016000200ED
:10451A00000000000001320000000000014B01F31E
:10452A00FFBFFF020100000000000132000000008E
:10453A000001FD009EFF740002000000000000015F
:10454A00320000000000015501F3FFBDFF02010027
:10455A000000000001320000000000011800030002
:10456A00F2FF02000000000000013200000000001B
:10457A0001FB001A00D5FF02010000000000013211
:10458A000000000000017B0030003800020000003B
:10459A0000000001320000000000018101B3FF01A8
:1045AA0000020100000000000132000000000001CA
:1045BA0086004F00F2FF02000000000000013200F6
:1045CA0000000000017C01B4FF00000201000000AD
:1045DA00000001320000000000017F004C000000D2
:1045EA00020000000000000132000000000001F497
:1045FA00001700D5FF020100000000000132000090
:10460A00000000015600F3FF320002000000000023
:10461A00000132000000000001ED001600D6FF0282
:10462A000100000000000132000000000001C40087
:10463A00ECFF7400020000000000000132000000DC
:10464A000000018101B3FF00000201000000000028
:10465A000132000000000001FD00580084FF020042
:10466A00000000000001320000000000016D01B7E7
:10467A00FF000002010000000000013200000000FB
:10468A000001E4004900740002000000000000017B
:10469A0032000000000001ED001600D6FF02010002
:1046AA000000000001320000000000015B00D3FF9F
:1046BA00E1FF0200000000000001320000000000DB
:1046CA00013D000A0007000201000000000001325B
:1046DA000000000000011600F4FF060002000000BE
:1046EA00000000013200000000000143000C00FA43
:1046FA00FF0201000000000001320000000000017A
:10470A001700F4FF07000200000000000001320059
:10471A00000000000147000200F2FF020100000051
:10472A00000001320000000000018500B1FF0D0009
:10473A000200000000000001320000000000013EFB
:10474A00000300F4FF020100000000000132000033
:10475A00000000017F0004004C000200000000007D
:10476A000001320000000000015001F3FFBEFF0209
:10477A0001000000000001320000000000010200F8
:10478A000000FFFF020000000000000132000000EC
:10479A0000000143000900F6FF02010000000000CA
:1047AA0001320000000000011600F7FF0A000200B3
:1047BA000000000000013200000000000124000691
:1047CA0000040002010000000000013200000000A5
:1047DA0000010D00FAFFFBFF0200000000000001CB
:1047EA003200000000000102011B00D4FF02010098
:1047FA000000000001320000000000010200000079
:10480A00FFFF02000000000000013200000000006B
:10481A000135000800F9FF02010000000000013222
:10482A00000000000001CB00EBFF7800020000004E
:10483A000000000132000000000001200005000411
:10484A000002010000000000013200000000000127
:10485A0082004E0000000200000000000001320049
:10486A00000000000141000B00F9FF0201000000F6
:10487A0000000132000000000001C30001008BFFAC
:10488A0002000000000000013200000000000139AF
:10489A0000080008000201000000000001320000C8
:1048AA0000000001AF0E3200CF0802010000000034
:1048BA0000013200000000000201000000000000B8
:1048CA00000000000000D8CFE4FFE0CFE4FFE46E70
:1048DA00E9CFE4FFEACFE4FFF3CFE4FFF4CFE4FF4C
:1048EA00E6528BEC34F0EFEC33F0030EDB6AA4A64D
:1048FA009DD1A4960E01002B0E01AB510E01005D55
:10490A0001E284D0006B0E01BAEC33F0EF6A7990C1
:10491A007B6A7A6A0E01A92B0E01AA510E01A95DC2
:10492A0001E3A96B83EC34F0EA22EE50ED106EE05D
:10493A0021EC35F0D5EC34F002E15750551847E038
:10494A0099EC34F0EA22EE50ED103AE0ACEC34F097
:10495A008FEC33F083EC34F0EA22EE50565C546E5E
:10496A00EE505758556E020E54C0DBFF030E55C069
:10497A00DBFF0EEC34F0553412E254500008000EFE
:10498A0055540DE20EEC34F099EC34F0BFEC34F0EF
:10499A0017E208EC35F0EE265550ED2218D00EEC51
:1049AA0034F0546C551E000E552299EC34F0BFECCD
:1049BA0034F006E208EC35F0EE5E5550ED5A07D0B9
:1049CA0021EC35F0EA2254C0EEFF55C0EDFFBAECF7
:1049DA0033F0120EEF6EF29E0E0183EC34F052ECBD
:1049EA0033F055C054F0556A5450B66E83EC34F027
:1049FA0052EC33F05450B56EF00EB4140009B46E94
:104A0A00F00EB4140909B46E7980F28E000ED880C3
:104A1A001F54000E20542EE22D2A000E2E221F5063
:104A2A002D5C20502E5826E32D6A2E6A030E235C35
:104A3A001FE22150EA6A200FE96E010EEA2280CFB6
:104A4A00EFFF2150EA6A230FE96E010EEA2281CFB5
:104A5A00EFFF2150EA6A260FE96E010EEA2282CFA1
:104A6A00EFFF212A030E215C01E3216A232A02D0E7
:104A7A001F6A206A000ED8802454000E25541CE2B6
:104A8A00000ED8803354000E345416E22F2A000E3A
:104A9A00302224502F5C255030580EE32F6A306A9A
:104AAA00030E285C07E2262A030E265C01E3266A27
:104ABA00282A02D0246A256A335034100BE0050EE6
:104ACA00325C07E3C18C9E9C9D8CC280C282326A92
:104ADA0001D0322A0501005101E1A4D0DE6ADD6A63
:104AEA00DECF54F0DDCF55F0040E545C000E55585D
:104AFA0001E398D058EC33F095EC33F0FDE1010E68
:104B0A00E926050EEA22EE50ED1070E058EC33F07B
:104B1A0095EC33F0FDE1D9EC34F0EE50ED1016E1EE
:104B2A00DEEC34F001E18180E2EC34F003E1ED5097
:104B3A0001E18182E6EC34F003E1ED5001E1818488
:104B4A00EAEC34F003E1ED5001E1818658EC33F0F0
:104B5A0095EC33F0FDE1B6EC34F095EC33F0FDE181
:104B6A00010EE926050ED5EC34F019E15750551817
:104B7A0016E1DEEC34F001E18190E2EC34F003E17D
:104B8A00ED5001E18192E6EC34F003E1ED5001E1F0
:104B9A008194EAEC34F003E1ED5001E1819658EC9E
:104BAA0033F095EC33F0FDE1D9EC34F0EE2A000E47
:104BBA00EF2258EC33F095EC33F0FDE1B6EC34F02B
:104BCA0095EC33F0FDE1090EE926050ED5EC34F03B
:104BDA0023E15750551820E158EC33F095EC33F0A7
:104BEA00FDE1D9EC34F0EE6AED6A16D0DEEC34F071
:104BFA0001E18190E2EC34F003E1ED5001E18192B0
:104C0A00E6EC34F003E1ED5001E18194EAEC34F092
:104C1A0003E1ED5001E18196DF2A010E01E260D73E
:104C2A00DB2A5ED70201F45101E0F4079EAC3BD0C7
:104C3A009E9CC1AC06D0C19C010E356E366A316AA3
:104C4A0017D0C450566E576E566AC350000156109C
:104C5A00546E57C055F03150E96EEA6ADFEC33F012
:104C6A0054C0EEFF55C0EDFFD89035363636312A9E
:104C7A00100E315C0EE235503314546E3650341433
:104C8A00556E5450551005E1312AD89035363636CE
:104C9A00EFD7100E315C02E39D9C05D03150040D14
:104CAA00F328C26EC282F2A433D0D59EF294F29A4D
:104CBA00040E546E2C50F5EC33F0EF50545C28E19E
:104CCA00080E2C5C0AE22AEC34F004E0E846FE0BFB
:104CDA005406FCE1E81C891616D0100E2C5C0AE278
:104CEA002AEC34F004E0E846FE0B5406FCE1E81C2A
:104CFA008A1609D02AEC34F004E0E846FE0B540682
:104D0A00FCE1E81C8B162C50F5EC33F0020EEF6E2A
:104D1A00040EE15C02E2E16AE552E16EE552E5CF9A
:104D2A00DAFFE7CFD9FFE552E5CFF4FFE5CFF3FF8E
:104D3A00E5CFEAFFE5CFE9FFE550E5CFE0FFE5CFB4
:104D4A00D8FF10000EEC35F0896A9268336A346A2B
:104D5A008A6A93688B6A94688C968C9495969594D3
:104D6A00928E0601010EFD6F0201FB69FC69276A3A
:104D7A00266A286A226A216A236A1F6A206A246AC2
:104D8A00256A2D6A2E6A2F6A306A316A768276809F
:104D9A00769C769A76887696FA0E776EDF6ADFCFF9
:104DAA004BF0100EE76E4B18E8AE02D0E73402D093
:104DBA00E7504B5C0BE2DFCFE9FFEA6AE9BEEA683B
:104DCA00DFEC33F0EE6AED6ADF2AE9D70601F76B0A
:104DDA00F86BF56BF66BF96BFA6BFB6BFC6B2A6A7B
:104DEA002B6A2C6ADF6ADFCF4BF0180EE76E4B187E
:104DFA00E8AE02D0E73402D0E7504B5C16E2DFCFD0
:104E0A00E9FFEA6AE9BEEA683FEC34F0EE6AED6A65
:104E1A00DFCFE9FFEA6AE9BEEA68290EE926010E50
:104E2A00EA22010EEF6EDF2ADED7D586D59AD59C07
:104E3A00F294F29AF1940F01498FBE0EC16ED08E90
:104E4A007694A386A5964AEC37F03AEC52F0F28EA5
:104E5A00F28C7684E552E55235EF33F00EEC35F0FC
:104E6A00EFEC33F0030EDB6A040EDB6A59EC32F026
:104E7A002350000809E284EC2CF0222A030E225C5B
:104E8A0001E1226A2306F4D72850000809E2A6ECB9
:104E9A002CF0272A030E275C01E1276A2806F4D79B
:104EAA00200E0601E76EA819E8AE02D0E73402D058
:104EBA00E750A85D01E231D16550020B01E02DD126
:104ECA00400EE66E400EE66E020EE66ED1EC50F033
:104EDA001DEC35F0E76E030EE7CFDBFFDB50000871
:104EEA0001E3E5D0040EDB6A030EDB50F36E040E19
:104EFA00E5EC33F001E3DBD0040EDB50EA6A400F45
:104F0A00E96E020EEA22EFCFDFFF05015D5132E1C1
:104F1A000D0E66EC33F005E00A0E4C6EDF504C5C69
:104F2A0029E1010E5D6F06019DEC33F00D0EEF6E67
:104F3A00F72B010EDB6AF751F36E010EE5EC33F045
:104F4A0014E236EC34F0E9BEEA68000EE926030EF4
:104F5A00EA22EF50E66E36EC34F0E9BEEA68190E42
:104F6A00E926050E4BEC34F0E6D734D90601F76B87
:104F7A00F86B8DD01B0EDF5C09E1595107E1010E78
:104F8A00596F1B0E5A6F5B6B5C6B81D059050BE135
:104F9A005B0EDF5C08E11B0E5A5D05E15B5103E124
:104FAA005B0E5B6F74D059054AE1410EDF5C47E145
:104FBA001B0E5A5D44E15B0E5B5D41E15A6B5B6B14
:104FCA005C6B596B010EDB6ADBCFE9FFEA6AE9BE6B
:104FDA00EA68000EE926030EEA22EF500D0814E0F3
:104FEA0036EC34F0E9BEEA68190EE926050EEA2223
:104FFA00EF50E66E36EC34F0E9BEEA68000EE926B8
:10500A00030E4BEC34F0E0D7010EDBCFF7F60601C6
:10501A009DEC33F0EF6A6C0E4B6EA00E7BEC34F015
:10502A00000EE66E030EE66E690E4B6EA00E88EC5D
:10503A0034F002E2E16AE552E16E4E5028D0080EE1
:10504A00DF5C0EE10601F75100080AE2F7079DEC62
:10505A0033F0EF6A660E4B6EA00E7BEC34F017D07D
:10506A000D0EDF5C14E00A0EDF5C11E0200EDF5C3F
:10507A000EE305015A6B5B6B5C6B596B06019DEC89
:10508A0033F0DFCFEFFF05015D6B0601F72B060159
:10509A00F7514B6E4C6A000E4B1806E1010E4C1884
:1050AA0003E12986F76BF86B040EDB2A1DD729501A
:1050BA0033E029A005D0600E4B6EA00E7BEC34F0D5
:1050CA0029A205D0410E4B6EA00E7BEC34F029A428
:1050DA0005D0250E4B6EA00E7BEC34F029A605D028
:1050EA00090E4B6EA00E7BEC34F029A805D0EA0E0F
:1050FA004B6E9F0E7BEC34F029AC05D0C90E4B6E7B
:10510A009F0E7BEC34F0000E291405E0B00E4B6EB6
:10511A009F0E7BEC34F0296A37D8050EE15C02E277
:10512A00E16AE552E16E35EF33F08BEC34F0F5C607
:10513A00DFFFDF2A400E66EC33F001E1DF6A060189
:10514A00F651DF5C01E120D80601F551EA6A000F49
:10515A00E96E020EEA22FD0EDBCFEFFFF52B400EC1
:10516A00F55D01E1F56BF651F55D01E12984FD0E6E
:10517A00DBCF4BF04C6A4BBE4C684BC0F3FF4CC0C4
:10518A00F4FFE55235EF33F08BEC34F00601F551BC
:10519A00F65D1DE00601905105E05BEC51F0BAECBA
:1051AA0041F0F8D70601F651D880F55507E2F651D5
:1051BA00F55D7DEC33F0F5C6F6F607D0400ED880E3
:1051CA00F6557DEC33F00601F66B5BEC51F0E552D7
:1051DA0035EF33F00EEC35F0E652E652DE6ADD6A60
:1051EA00020EDB6A030EDB6A060145EC33F052EC71
:1051FA0034F0020EF3CFDBFF06015FEC33F004E17B
:10520A00010E4C1801E1F86B020EDB50DE6EDD6A0E
:10521A0045EC33F02C0824E045EC33F00D0820E08F
:10522A0045EC33F052EC34F0030EF3CFDBFF06010A
:10523A005FEC33F004E1010E4C1801E1F86B020E49
:10524A00DBCF4DF04DC04EF04D6A030EDB5000012E
:10525A004D244B6E000E4E204C6E4BC0DEFFDD6EB1
:10526A00000EDFCF3DF0010EDBCF3EF04D0E3D18B4
:10527A0002E1580E3E1801E1E3D1530E3D1802E156
:10528A00450E3E1801E1D9D1430E3D1802E1410E07
:10529A003E1801E1D0D14D0E3D1802E1510E3E18E3
:1052AA0001E1C6D14D0E3D1802E1520E3E1801E150
:1052BA00BCD1320E3D1802E1530E3E1801E1B2D1C3
:1052CA00450E3D1802E1530E3E1801E1A8D1430EE6
:1052DA003D1802E1510E3E1801E19ED14B0E3D18D8
:1052EA0002E1430E3E1801E194D14C0E3D1802E151
:1052FA00420E3E1801E18AD1440E3D1802E14E0EDB
:10530A003E1801E180D1490E3D1802E14E0E3E18C9
:10531A0001E176D1420E3D1802E1510E3E1801E13B
:10532A006CD14C0E3D1802E1510E3E1801E162D1DA
:10533A004C0E3D1802E1530E3E1801E158D14E0EB3
:10534A003D1802E1510E3E1801E14ED14E0E3D18B4
:10535A0002E1530E3E1801E144D1430E3D1802E129
:10536A00530E3E1801E13AD14D0E3D1802E1450EA9
:10537A003E1801E130D1500E3D1802E1510E3E189F
:10538A0001E126D1500E3D1802E1540E3E1801E10A
:10539A001CD1500E3D1802E1530E3E1801E112D104
:1053AA004D0E3D1802E1530E3E1801E108D1470E99
:1053BA003D1802E1500E3E1801E1FED0430E3D18A1
:1053CA0002E1500E3E1801E1F4D0490E3D1802E107
:1053DA00430E3E1801E1EAD0490E3D1802E1520E91
:1053EA003E1801E1E0D0490E3D1802E1530E3E1885
:1053FA0001E1D6D0530E3D1802E1430E3E1801E1F9
:10540A00CCD0530E3D1802E1520E3E1801E1C2D033
:10541A00530E3D1802E1530E3E1801E1B8D0530E67
:10542A003D1802E1420E3E1801E1AED0430E3D188E
:10543A0002E1420E3E1801E1A4D0430E3D1802E1FA
:10544A00520E3E1801E19AD04F0E3D1802E1420E6B
:10545A003E1801E190D0570E3D1802E14D0E3E185C
:10546A0001E187D0520E3D1802E14D0E3E1801E1CE
:10547A007ED0440E3D1802E1500E3E1801E175D06F
:10548A004F0E3D1802E1500E3E186DE0490E3D18D0
:10549A0002E1500E3E1865E0580E3D1802E1540E26
:1054AA003E185CE0540E3D1801E13E5055E0410EB5
:1054BA003D1801E13E504EE0560E3D1801E13E50C6
:1054CA0047E0490E3D1801E13E5040E04F0E3D18BD
:1054DA0001E13E5039E0550E3D1802E1430E3E18F7
:1054EA0031E0580E3D1802E1430E3E1828E0430E03
:1054FA003D1801E13E5021E0520E3D1801E13E50B7
:10550A001AE0580E3D1802E1520E3E1811E0030E41
:10551A00DB5001E098D0020EFFEC33F0FFEC33F0E1
:10552A008D0E4B6E9F0EB1EC34F001E39BD098D0F8
:10553A00D5EC2EF099D0BDD897D00CD995D0D7EC10
:10554A002EF092D0BAD890D0A6D98ED0D8D98CD0F5
:10555A00F3D98AD0F6D988D0D4D886D0D3EC2EF015
:10556A0083D014DB81D085DB7FD07BDA7DD059DA1A
:10557A007BD045DA79D048EC2FF076D0D9EC2EF0F2
:10558A0073D046EC2FF070D04AEC2FF06DD04CEC73
:10559A002FF06AD04EEC2FF067D050EC2FF064D089
:1055AA0052EC2FF061D054EC2FF05ED056EC2FF075
:1055BA005BD058EC2FF058D0B0EC2FF055D0C5EC9A
:1055CA0038F052D009EC3CF04FD0ECEC3BF04CD028
:1055DA00DAEC3BF049D08AEC3CF046D001EC38F0EA
:1055EA0043D007EC3DF040D026EC3DF03DD037ECFF
:1055FA003DF03AD043EC3DF037D054EC3DF034D096
:10560A00E9EC3CF031D0FAEC3CF02ED0E5EC2FF08E
:10561A002BD0EDEC2FF028D067EC3DF025D07AECBA
:10562A003DF022D0B1EC52F01FD0E4EC3DF01CD09A
:10563A00E5EC3DF019D01BD917D059EC3BF014D04A
:10564A005CEC39F011D0C5EC34F0C5EC34F0650EE1
:10565A004B6E9F0E26EC33F04E6E0B0EE15C02E2AF
:10566A00E16AE552E16E4E50060145EC33F00D0851
:10567A000DE029500BE1520E4B6E4C6ADF504B186D
:10568A0003E1DE52DD504C1801E0298EF7C6F8F628
:10569A00040EE15C02E2E16AE552E16E35EF33F0B5
:1056AA000601FD5105E0400E4B6EAD0E7BEC34F069
:1056BA001200A7EC26F055EF2BF08BEC34F003EC3C
:1056CA0035F040EC33F0020E23EC33F0295017E1A9
:1056DA00DF0414E1D950010F59EC34F00AE0010E4D
:1056EA004B6E4C6ADB504B1808E1020EDB504C182B
:1056FA0004E1010EDBCFFDF601D0298CD1DF8EEF5C
:10570A0034F02FEC33F0EFEC33F0E66A1D0EE66E60
:10571A00000EE66E25EC35F01BE1020EDB500CE1C3
:10572A001D501E1003E11F6A206A11D076841DC025
:10573A001FF01EC020F00BD01D501E1003E1246A7A
:10574A00256A05D076841DC024F01EC025F0A8DF86
:10575A008EEF34F00EEC35F0E65203EC35F035EC12
:10576A0035F0020F35EC35F0030F35EC35F0040F48
:10577A007EEC34F00FE1DF50926E010EDB50936E37
:10578A00020EDB50946E030EDB50956E040EDB5056
:10579A00966E86DF050EE15C02E2E16AE552E16E91
:1057AA0035EF33F02FEC33F0FD0EDB50100805E235
:1057BA00100EF36EFD0EF3CFDBFFFC0EDB5029E07B
:1057CA00FD0EDB50E7EC56F0F3503312F45034126E
:1057DA00080EF36EFD0EE5EC33F00DE2010EF36EEA
:1057EA00FD0EDB5003E05BEC33F0FDE1F350F31CFC
:1057FA000F0148173AD0FD0EDB500C0836E35DEC7A
:10580A0034F003E03BEC34F0FDE1E81C0F014917EA
:10581A002CD0FD0EDB50E7EC56F0F3CF4BF0F4CF73
:10582A004CF04B1E4C1E4B5033164C503416080E7F
:10583A00F36EFD0EE5EC33F00CE2010EF36EFD0E95
:10584A00DB5003E05BEC33F0FDE1F3500F0148134A
:10585A000CD0FD0EDB500C0808E35DEC34F003E0DD
:10586A003BEC34F0FDE10F01491335EF33F02FEC37
:10587A0033F003EC35F07EEC34F009E1010EDBCFB6
:10588A00E6FFDFCFE6FF8EDFE552E55209DFE5529C
:10589A00E55235EF33F02FEC33F04EEC33F0010ED6
:1058AA0023EC33F0AEEC33F026E1010EDB5002E1DB
:1058BA00DF50896E95EC34F01EE1010EDB5002E1F7
:1058CA00DF508A6E95EC34F016E1010EDB5002E1EE
:1058DA00DF508B6E95EC34F00EE1010EDB5002E1E5
:1058EA00DF508C6E95EC34F006E1010EDB5002E1DC
:1058FA00DF508D6ED5DEE552E55235EF33F0845038
:10590A00E66EE66A8350E66EE66A8250E66EE66AFC
:10591A008150E66EE66A8050E66EE66A480E4B6E85
:10592A009F0E26EC33F04E6E0D0EE15C02E2E16A48
:10593A00E552E16E4E501200480E4B6EAD0E7BEFF3
:10594A0034F00EEC35F0E652DF6A010EF36EDB6ED0
:10595A00020EDB6A460E4B6E9F0E7BEC34F09DBC4A
:10596A00FED7DF6ADFCF4BF0100EE76E4B18E8AEBA
:10597A0002D0E73402D0E7504B5C3AE2010EDB502A
:10598A0033144B6E020EDB5034144C6E4B504C10D9
:10599A001EE0DFCFE9FFEA6AE9BEEA68DFEC33F02E
:1059AA00EECFE6FFEFCFE6FFDFCF4BF04C6A4BBE00
:1059BA004C68EEEC34F03B0E4D6E9F0E03EC34F067
:1059CA00070EE15C02E2E16AE552E16E5050010E17
:1059DA00DBCF4BF0020EDBCF4CF0D8904B364C3677
:1059EA00010E4BC0DBFF020E4CC0DBFFDF2ABAD729
:1059FA00450E4B6EAD0E7BEC34F08EEF34F08BEC33
:105A0A0034F04EEC33F025EC35F009E121EC34F0BA
:105A1A0005E2F3EC34F0020EDBCFEFFF41DE8EEF4E
:105A2A0034F08BEC34F04EEC33F0030E23EC33F00D
:105A3A00295015E121EC34F005E2F3EC34F0020EC2
:105A4A00EFCFDBFF020EFFEC33F0310E4B6E9F0EF1
:105A5A0088EC34F002E2E16AE552E16E4E508EEFD4
:105A6A0034F039EC35F001E08FD0020EDB5001083A
:105A7A0001E287D0010EDB50070801E282D0410E15
:105A8A0066EC33F016E1020EDB500AE16AEC33F001
:105A9A0003E05BEC33F0FDE1F350F31C921673D094
:105AAA006AEC33F003E05BEC33F0FDE1F350921261
:105ABA006AD0420E66EC33F016E1020EDB500AE1C0
:105ACA006AEC33F003E05BEC33F0FDE1F350F31CD6
:105ADA00931659D06AEC33F003E05BEC33F0FDE146
:105AEA00F350931250D0430E66EC33F016E1020ED7
:105AFA00DB500AE16AEC33F003E05BEC33F0FDE1E2
:105B0A00F350F31C94163FD06AEC33F003E05BECDD
:105B1A0033F0FDE1F350941236D0440E66EC33F0C4
:105B2A0016E1020EDB500AE16AEC33F003E05BECAB
:105B3A0033F0FDE1F350F31C951625D06AEC33F0EF
:105B4A0003E05BEC33F0FDE1F35095121CD0450EF7
:105B5A0066EC33F016E1020EDB500AE16AEC33F030
:105B6A0003E05BEC33F0FDE1F350F31C96160BD027
:105B7A006AEC33F003E05BEC33F0FDE1F35096128C
:105B8A0002D0298C01D08CDD8EEF34F02FEC33F06B
:105B9A00EFEC33F02FEC35F0050E77EC34F0010F13
:105BAA007EEC34F064E1010EDB5007084CE3410E51
:105BBA0066EC33F00AE1B4EC33F003E03BEC34F08A
:105BCA00FDE1E8407F0B801437D0420E66EC33F0DB
:105BDA000AE1B4EC33F003E03BEC34F0FDE1E840D9
:105BEA007F0B811429D0430E66EC33F00AE1B4EC42
:105BFA0033F003E03BEC34F0FDE1E8407F0B821424
:105C0A001BD0440E66EC33F00AE1B4EC33F003E047
:105C1A003BEC34F0FDE1E8407F0B83140DD0450ED8
:105C2A0066EC33F010E1B4EC33F003E03BEC34F013
:105C3A00FDE1E8407F0B8414E76E020EE7CFDBFF3D
:105C4A00DB5008E002D0298C12D0010EF36E020E4E
:105C5A00F3CFDBFF020EFFEC33F0280E4B6E9F0EE4
:105C6A0088EC34F002E2E16AE552E16E4E508EEFC2
:105C7A0034F039EC35F001E08FD0020EDB50010828
:105C8A0001E287D0010EDB50070801E282D0410E03
:105C9A0066EC33F016E1020EDB500AE16AEC33F0EF
:105CAA0003E05BEC33F0FDE1F350F31C891673D08B
:105CBA006AEC33F003E05BEC33F0FDE1F350891258
:105CCA006AD0420E66EC33F016E1020EDB500AE1AE
:105CDA006AEC33F003E05BEC33F0FDE1F350F31CC4
:105CEA008A1659D06AEC33F003E05BEC33F0FDE13D
:105CFA00F3508A1250D0430E66EC33F016E1020ECE
:105D0A00DB500AE16AEC33F003E05BEC33F0FDE1CF
:105D1A00F350F31C8B163FD06AEC33F003E05BECD4
:105D2A0033F0FDE1F3508B1236D0440E66EC33F0BB
:105D3A0016E1020EDB500AE16AEC33F003E05BEC99
:105D4A0033F0FDE1F350F31C8C1625D06AEC33F0E6
:105D5A0003E05BEC33F0FDE1F3508C121CD0450EEE
:105D6A0066EC33F016E1020EDB500AE16AEC33F01E
:105D7A0003E05BEC33F0FDE1F350F31C8D160BD01E
:105D8A006AEC33F003E05BEC33F0FDE1F3508D1283
:105D9A0002D0298C01D084DC8EEF34F055EF2BF041
:105DAA0055EF2BF055EF2BF00EEC35F0FDEC34F0FF
:105DBA00BCEC34F05FE1D950020FF8EC34F0720E0B
:105DCA00D880EE542E0EED543BE3D950020F59EC15
:105DDA0034F01FE04E684F68506A2D0EE76E020ECF
:105DEA00DBCF51F0030EDBCF52F0E7505126000E05
:105DFA005222536A51504E5C4B6E52504F584C6E61
:105E0A00535050584D6E020E4BC0DBFF030E4CC070
:105E1A00DBFF010EDB50070813E3410E66EC33F09B
:105E2A0002E1DF6A0FD0420E66EC33F002E1080E9F
:105E3A0005D0430E66EC33F003E1100EDF6E02D09C
:105E4A00298C18D0010EDB50DF24E96EEA6A3FEC98
:105E5A0034F064EC34F0010EDB50DF24F5EC33F05F
:105E6A00EF0407E1010EDB50DF24F5EC33F0020EFC
:105E7A00EF6E16DC040EE15C02E2E16AE552E16EC5
:105E8A00EFD355EF2BF055EF2BF055EF2BF055EFE5
:105E9A002BF055EF2BF055EF2BF055EF2BF055EF7C
:105EAA002BF055EF2BF0D6DB070EE12402E3E16875
:105EBA00E652E16E2FEC35F0030E77EC34F0BCECD1
:105ECA0034F042E1DECF01F5DDCF02F5020EDBCF81
:105EDA0009F5030EDBCF0AF5040EDB6A030EF36E37
:105EEA00040EE5EC33F02EE28BEC33F0030EA6DB66
:105EFA00E76E050EE7CFDBFF010EE66ED9502AECFE
:105F0A0035F0E76E060EE7CFDBFF29501DE1050EDF
:105F1A00DB5018E1060EDB5015E145EC34F0010EBA
:105F2A00E926050EEA22DECFEEFFDDCFEDFF45ECD6
:105F3A0034F0090EE926050EEA2264EC34F0040E68
:105F4A00DB2ACCD755EC2BF0070EE15C02E2E16AC2
:105F5A00E552E16E85D38BEC34F02FEC35F0010E6F
:105F6A006DDB29500DE1DF5007E0F00E9314936EBC
:105F7A000501010E006F02D00501006B55EC2BF0F4
:105F8A00E5526ED3D9CFE6FFDACFE6FFE1CFD9FFEC
:105F9A00E2CFDAFFE652DF6AFF0EDF5C0AE2E86868
:105FAA00E85005E0E80600D000D000D0F9D7DF2A93
:105FBA00F3D7E552E552E5CFDAFFE7CFD9FF120072
:105FCA00F29EF29C6592656ADDDF0FEF00F0120027
:105FDA0041DB100EE12402E3E168E652E16EE66A73
:105FEA00D950010F48DBE66ACAEC34F02FEC35F0E1
:105FFA00010E77EC34F0040F3EDB020E77EC34F03E
:10600A00020F39DB030E77EC34F00A0F34DB060E8D
:10601A0077EC34F0060F2FDB070E77EC34F00E0F17
:10602A002ADB040E77EC34F00F0F25DB050E06DBB6
:10603A00010EDBCF4BF04C6A4BBE4C68EEEC34F0F1
:10604A001C0E4D6E9F0EDADB050EE15C02E2E16A80
:10605A00E552E16E5050DFCFE6FFE66A100E4B6E56
:10606A009F0E88EC34F002E2E16AE552E16E4E508E
:10607A00040EDBCFE6FF050EDBCFE6FF040E4B6E08
:10608A009F0E88EC34F002E2E16AE552E16E4E506E
:10609A00020EDBCFE6FF030EDBCFE6FFF80E4B6EF8
:1060AA009E0E88EC34F002E2E16AE552E16E4E504F
:1060BA00D9500A0F68DBEB0E4B6E9E0EB1EC34F032
:1060CA0002E2E16AE552E16E4E50D950060F5BDBFF
:1060DA00DE0E4B6E9E0EB1EC34F002E2E16AE5523E
:1060EA00E16E4E500E0E86DBD20E4B6E9E0E88EC83
:1060FA0034F002E2E16AE552E16E4E500F0E7ADBAD
:10610A00C60E4B6E9E0E88EC34F002E2E16AE5524E
:10611A00E16E4E5055EC2BF0100EE15C02E2E16AA2
:10612A00E552E16E9DD296DA090EE12402E3E168B6
:10613A00E652E16E080EDB6A0D0E4B6E0601A0DA1E
:10614A004B5C05E1FA0EDB5026E1298824D098DA67
:10615A002C0812E0FA0EDB500DE192DAE66EE66ADE
:10616A009F0E4B6E9E0ECFDB02E2E16AE552E16EB4
:10617A004E50298A020E21D19DDA04E1010E4C18F3
:10618A0001E1F86B0D0E4B6E7BDA4B5C06E1FA0E01
:10619A00DB5001E12988030E10D12D0E4B6E70DA07
:1061AA004B5C20E1040E43DB1DE0050E4D6EFD0E37
:1061BA00DB504D5C17E0FD0EDB0401E1C4D0030E99
:1061CA0004DB01E1C0D0070E32DB01E1BCD0010ED5
:1061DA00F36E080EF3CFDBFF6DDA04E1010E4C1803
:1061EA0001E1F86B040EF1DA0AE0050E20DB07E0A4
:1061FA000A0EE66E90DBEAD81DEC35F036D0F8517F
:10620A0098DBEFCF4BF0000E4BC0DFFF010EDB6ACD
:10621A00020EDB6A030EDB6A050ED7DA1FE1000EF7
:10622A00DFCFE6FF010EDBCFE6FF56EC56F0E55274
:10623A00E552F3CF4BF0F4CF4CF04D6A4E6A4CAEB8
:10624A0002D04D684E684BC0DFFF010E4CC0DBFF29
:10625A00020E4DC0DBFF030E4EC0DBFF06012ADA39
:10626A0004E1010E4C1801E1F86B080EDB503FE027
:10627A00FD0EDB5006E1F1DB800E34DA000EEE543F
:10628A0062E3020EA2DA06E1E8DB000EEE54800EAB
:10629A0029DA59E3060ECBDA06E1DFDB000E22DA51
:1062AA00800EEE5450E3F0D978DA080EDB5053E052
:1062BA00040EDBCF3BF0050EDBCF3CF0060EDBCF46
:1062CA003DF0070EDBCF3EF0406841684268436804
:1062DA00F1EC55F0040E37C0DBFF050E38C0DBFFCA
:1062EA00060E39C0DBFF070E3AC0DBFF34D0FD0EC5
:1062FA00DB5006E1B2DB7F0EEE54000EF3D923E346
:10630A00FD0EDB0404E11BDB000EECD91CE3020EDC
:10631A005CDA04E114DB7F0EE5D915E3030E87DAB4
:10632A0004E10DDBFF0EDED90EE3060E4D6EFD0E07
:10633A00DB504D5C0BE103DBFF0EEE54FF0EEE5417
:10634A007F0EEE5403E2298C010E37D0070E3DDA98
:10635A0002E09AD922DAFD0EDB50070A21E0010A8F
:10636A0017E0050A11E0010A0FE0030A08E0050A2E
:10637A0006E0010A04E0050A02E0040E1ED0DBD999
:10638A00040EDBCFEFFF18D005DBDBCFEDFF14D017
:10639A0001DBDBCFEEFF060EDBCFEEFF070E0AD0E6
:1063AA00CAD9DFCFEEFF010EDBCFEEFF020EDBCF45
:1063BA00EEFF030EDBCFEEFF000E4B6E090EE15C23
:1063CA0002E2E16AE552E16E4B504AD122DB28DA59
:1063DA00EE6AEE6AEE6AEE6A010EDB6AFB0EDB50CB
:1063EA00F36E010EEDD94FE20601F851A2DAEFCFB2
:1063FA00DFFF300EDF5C42E3DF5039083FE310DA9B
:10640A00EECF4BF0EECF4CF0EECF4DF0EFCF4EF09B
:10641A000A0E406E416A426A436A4BC03BF04CC066
:10642A003CF04DC03DF04EC03EF0F1EC55F037C0A7
:10643A004BF038C04CF039C04DF03AC04EF0300E37
:10644A00DF5C4F6E506A516A526AE8504B265050D0
:10645A004C2251504D2252504E22E2D94BC0EEFFEF
:10646A004CC0EEFF4DC0EEFF4EC0EEFF060122D932
:10647A0007E1010E4C1804E1F86B02D0000E04D0BB
:10648A00010EDB2AABD7010EE552E552E9D02350C3
:10649A00E66EE66A930E4B6E9E0E35DA02E2E16A0A
:1064AA00E552E16E4E5012000601A85108E0010EB5
:1064BA004B6E6550020B01E0010E4B5C17E1CBD924
:1064CA000BE16151621111E18C86A00E616F0F0E12
:1064DA00626F010E636F12006151621152E18C9674
:1064EA00A00E616F0F0E626F636B1200A80509E0C0
:1064FA00020EA85D06E0040EA85D03E0100EA85D7A
:10650A0017E1A9D90BE16151621111E18C86200EC4
:10651A00616F4E0E626F010E636F1200615162115C
:10652A0030E18C96200E616F4E0E626F636B120023
:10653A00200EA85D26E18FD907E16151621121E1A0
:10654A008C86CBD9010E15D0630507E16151621122
:10655A0018E18C96C2D9020E0CD0020E635D0BE1D3
:10656A00615162110EE18C86A00E616F860E626F18
:10657A00030E636F12006151621103E18C96ADD96B
:10658A00636B120067D8A2D9E8AE02D04B3403D0AD
:10659A00E750D8804B5423E3FC0EDB5010E0C3D8FD
:1065AA00E9BEEA6896D804E0E846FE0B4C06FCE130
:1065BA004B6EB9D8E9BEEA682FDAEF1210D0B3D819
:1065CA00E9BEEA6886D804E0E846FE0B4C06FCE120
:1065DA00E81C4B6EA8D8E9BEEA681EDAEF1640D06E
:1065EA0039D874D9E8AE02D04B3403D0E750D880FA
:1065FA004B5423E3FC0EDB5011E195D8E9BEEA685F
:10660A0068D804E0E846FE0B4C06FCE1E81C4B6E39
:10661A008AD8E9BEEA6806DAEF160FD084D8E9BE4E
:10662A00EA6857D804E0E846FE0B4C06FCE14B6EDC
:10663A007AD8E9BEEA68F6D9EF1212D0E66ECAEF46
:10664A0034F04C6E4D6A4BC0E6FFE66E4DC0E6FF75
:10665A001BEF55F060D9E1CFD9FFE2CFDAFF120084
:10666A00E552E5CFDAFFE7CFD9FF1200A951E96E6B
:10667A00EA6AA8EF34F0E66E000EDA20E66E12003F
:10668A00F85157D9EF501200D9CFE9FFDACFEAFF14
:10669A001200E652E6522FEF35F0EA22EECF54F01E
:1066AA00EFCF55F012009AD9010E1200D890F336A6
:1066BA00E8061200F82BF8514B6E4C6A000E4B1884
:1066CA0012004B6EDF504B5C1200010EF36EDB5072
:1066DA001200C80EE926050EEA22EF504C6E010E92
:1066EA004C521200EE54000EEE54000EEE541200FC
:1066FA00DF6EDFCFE6FFF6514C6A000F4B6E020EDB
:10670A004C2267D914EC51F01DEF35F0010EE66EFC
:10671A0090EF34F0EA22EECF56F0EFCF57F01200A6
:10672A0012D9E8061200FD0EDBCFE9FFEA6A120071
:10673A00F7519EEF34F0FB0EDBCFE9FFFC0EDBCF07
:10674A00EAFF1200EA22EE50EFCFEAFFE96E4B5061
:10675A001200E76E010EE7CFDBFF29501200010E8F
:10676A00DB284B6E010E4B521200A951EA6A310F17
:10677A00E96E0E0EEA22EF500E01EA6AAC25E96EC6
:10678A00AD51EA2212002FD9EECFE6FFEECFE6FF97
:10679A00EECFE6FFEFCFE6FF1200040EEECFDBFFEF
:1067AA00050EEECFDBFF060EEECFDBFF070EEECFB8
:1067BA00DBFF1200C8D8000EE926010EEA221200F9
:1067CA00DBCFF4FFF350F45C12004B6EFD0EDB508E
:1067DA004B5C1200E652E652E652020EDB6A1200E7
:1067EA00EA6A290FE96E010EEA2212004E6E050EC0
:1067FA00E15C1200DBCFE6FFE66A12004E6E4F6ADA
:10680A004DC0E6FFE66E4FC0E6FF1BEC55F0506E3A
:10681A001200020EDBCF54F0030EDBCF55F012004C
:10682A00FC0EDBCFE9FFFD0EDBCFEAFF12004C6E58
:10683A00FD0EDB504C5C1200DECF4BF0DDCF4CF08E
:10684A00000E4B5C100E4C581200070E2C14546E9E
:10685A00010E5452120005016107000E625B63517A
:10686A001200010EDBCFE9FFEA6A1200E846FE0BCE
:10687A004B06120068D8410EE926010EEA221200E0
:10688A00040EDB28E96EEA6AA8EF34F0EA22E55240
:10689A00E750EF6E010EDB2A1200E66EE66A56EC4E
:1068AA0056F0E552E55212009ED8EE50ED10120055
:1068BA00FD0EDB50F80F4B6E010E4B521200020E0A
:1068CA00DBCFEEFF030EDBCFEDFF1200FD0EDBCFB9
:1068DA004BF0190EE76E4B181200100E616F270E5F
:1068EA00626F1200ABDEE66AD9501200AADE1DEF13
:1068FA0035F0C1DE010EA2DE29501200B7DE010E0C
:10690A00E9260E0E12009DDEFBEF33F0A3DEE652FF
:10691A0012008ED8A5D6D9CFE6FFDACFE6FF12004D
:10692A00F5DE8CDEAEEF33F0A1DE790EE9260E0E2F
:10693A001200EA6A000FE96E030EEA2212008DD8ED
:10694A00FF0EEE541200D890E936EA3612008EDEB7
:10695A00490EE9260E0E120074DE4E6E070EE15C39
:10696A001200110EE926050E98DE58EF33F06DD8A5
:10697A0029501200CFDE5450565C55505758120019
:10698A00030E38DF020EFFEF33F098EC30F050D8E8
:10699A00E5521200D0DE040EDBCFEEFF050E120028
:1069AA00B9DE565054181200110EE926050EEA22D5
:1069BA0012006ADEEE50ED10120066DE010EEE18CD
:1069CA00120062DE020EEE1812005EDE030EEE18F0
:1069DA0012004BC0E6FF4CC0E6FF1200DECFE9FF13
:1069EA00DDCFEAFF1200E96E000EDA20EA6E12002D
:1069FA0050DE050E77DF010F35EF35F04ADE010E66
:106A0A0071DF010F120090DF48DE78DFEA2254506E
:106A1A0012007CDFE652120096DF960EE926050E7A
:106A2A00A7EF33F090DF640EE926050EA7EF33F0E7
:106A3A00E552E552E55212008ADF2FDE83EF34F089
:106A4A00030E50DF020F7EEF34F0020F14DE030E46
:106A5A0023EF33F0E66A90EF34F016DED8801200A6
:106A6A000ADE010E77EF34F051DFC2DF020F7EEF4C
:106A7A0034F0E9CFE4FFEACFE4FFE652D9CFE6FFEC
:106A8A00DACFE6FFE1CFD9FFE2CFDAFFE6529EA0E6
:106A9A00F0D19E908E0ECE6ECF680DC080F20201AC
:106AAA00816B0201010E826F0E500F10101011102F
:106ABA0014E0D880000E0E54000E0F54190E105414
:106ACA00000E115405E20E6A0F6A106A116A05D0A7
:106ADA000E06000E0F5A105A115A0E500F101010AF
:106AEA00111002E00201826B8392000401E0B3D02C
:106AFA00055006100710081006E109500A100B107D
:106B0A000C1001E1A7D00201EB510BE10DA202D05A
:106B1A008C8E01D08C9E0DA602D08C8A01D08C9AC4
:106B2A000DD00201EB050AE10DA202D08B8401D03F
:106B3A008B940DA602D0898401D089940550061041
:106B4A000710081023E018500124186E195002206B
:106B5A00196E000ED8801854800E195415E218C008
:106B6A0018F019C019F0000E185E800E195A010E9D
:106B7A00020180110201806F0201010E816F050678
:106B8A00000E065A075A085A0201826B09500A1067
:106B9A000B100C1023E01A5003241A6E1B50042009
:106BAA001B6E000ED8801A54800E1B5415E21AC0B0
:106BBA001AF01BC01BF0000E1A5E800E1B5A040E40
:106BCA00020180110201806F0201010E816F090624
:106BDA00000E0A5A0B5A0C5A0201826B02018151A9
:106BEA0039E00201EB5107E1020180B18C8C02010C
:106BFA0080B58C8809D00201EB0506E1020180B15B
:106C0A008B8C020180B5898A000000000000000018
:106C1A00000000000000000000000000000000006A
:106C2A00000000000000000000000000000000005A
:106C3A000000000000000000000000000000020147
:106C4A00EB5103E18C9C8C9805D00201EB0502E123
:106C5A008B9C899A9DD0030E005C01E099D00201B9
:106C6A00F85101E177D01504DF6E1250131037E1A5
:106C7A00DF50EA6A310FE96E0E0EEA22EF500E017A
:106C8A00EA6AAC25E96EAD51EA22EF6AEA6ADF34B4
:106C9A00FE0BEA36E96E790EE9260E0EEA22EE6A54
:106CAA00ED6AEA6ADF34FE0BEA36E96E490EE92636
:106CBA000E0EEA22EE6AED6ADF50EA6A310FE96ED9
:106CCA000E0EEA22EF6AEA6ADF34FE0BEA36E96E52
:106CDA00010EE9260E0EEA22EE6AED6A3BD0EA6A56
:106CEA00DF34FE0BEA36E96E790EE9260E0EEA2249
:106CFA0016C0EEFF17C0EDFFEA6ADF34FE0BEA3674
:106D0A00E96E490EE9260E0EEA2212C0EEFF13C002
:106D1A00EDFFDF50EA6A310FE96E0E0EEA2214C067
:106D2A00EFFFEA6ADF34FE0BEA36E96E010EE92666
:106D3A000E0EEA22EE50ED100DE1EA6ADF34FE0B88
:106D4A00EA36E96E010EE9260E0EEA2212C0EEFFBD
:106D5A0013C0EDFF0E01B651145C1AE10E01B051D9
:106D6A00121802E1B15113180AE10201010EEC6F87
:106D7A000201E86B0201F75101E08A9809D0020189
:106D8A00EC6B0201010EE86F0201F75101E08A88FB
:106D9A000201825162E00E500F10101011105DE1D5
:106DAA00006A1C5056E184C200F085C201F086C216
:106DBA0002F087C203F088C204F089C205F08AC2D1
:106DCA0006F08BC207F08CC208F08DC209F08EC2A1
:106DDA000AF08FC20BF090C20CF091C20DF092C271
:106DEA000EF093C20FF094C210F095C211F096C241
:106DFA0012F097C213F098C214F099C215F09AC211
:106E0A0016F09BC217F00201846B0201856B866B38
:106E1A000201876B886B0201896B8A6B8B6B8C6BA7
:106E2A0002018D6B8E6B8F6B906B0201916B02016D
:106E3A00926B936B946B956B0201966B976B020145
:106E4A00986B0201996B02019A6B9B6B010E1C6E87
:106E5A0004D00E6A0F6A106A116A8050800B06E02D
:106E6A000201F35106E08150010B03E10201010E18
:106E7A00F26FE552E552E5CFDAFFE7CFD9FFE552E7
:106E8A00E5CFEAFFE5CFE9FF1100D9CFE6FFDACF78
:106E9A00E6FFE1CFD9FFE2CFDAFFE652DF6ADFCFC2
:106EAA004BF0020EE76E4B18E8AE02D0E73402D080
:106EBA00E7504B5C24E2DFCFE9FFEA6AE9BEEA6801
:106ECA00D890E936EA36010EE926000EEA22010ECA
:106EDA00EE6EED6ADFCFE9FFEA6AE9BEEA68D890AA
:106EEA00E936EA36D890E936EA36050EE926000E82
:106EFA00EA22EE6AEE6AEE6AEE6ADF2AD0D7006A02
:106F0A000D6A0E6A0F6A106A116A126A136A146AA3
:106F1A00156A166A176A010E1C6ECD92CD9ECD9C1B
:106F2A00CD8ACD98CD96CD948E0ECE6ECF68CD807B
:106F3A009F809E909D8092809F9C010EE66EE66ADD
:106F4A00D7EC2BF0E552E552010EE66E0B0EE66E1B
:106F5A00D7EC2BF0E552E5528D8496948D82969269
:106F6A00898C929C8D8096908B8294928C9C959C15
:106F7A008C9E959E8C9895988C9A959A949E828EC2
:106F8A0000000000000000000000000000000000F7
:106F9A0000000000000000000000000000000000E7
:106FAA00000000000000948E829E0201010EF76F1D
:106FBA000201010EF86F8A9893980201010EE86F98
:106FCA000201EB6B0201010EEC6F0201F16B02018F
:106FDA00ED6BEE6BEF6BF06B0201F26B9380F19E3F
:106FEA000201010EF36F93968196E552E552E5CFC1
:106FFA00DAFFE7CFD9FF1200B6EC3EF08BEC3FF098
:10700A0058EC3FF04DEC41F0E66AD9503BEC41F0C8
:10701A00295001E0B3D0DF0424E14BEC3FF00CE14E
:10702A000201010EF76FF86B7CEC3FF002E2E16AB5
:10703A00E552E16E4B500DD0D8EC3FF006E1ED5031
:10704A0004E10201F76B010E03D00201010EF76F92
:10705A00F86F000EE66EE66AECC2E6FFEEEC3FF071
:10706A008BD0020EDF5C2EE14BEC3FF009E102010E
:10707A00EB6B96909492959C959E9598959A1BD0B9
:10708A00D8EC3FF00DE1ED500BE10201010EF0ECFE
:10709A003FF094949294949C929A959292926CD086
:1070AA002AEC41F0020EEE1867E1ED5065E10201AB
:1070BA00020EF0EC3FF094849284948C928A95822A
:1070CA0092825AD0040EDF5C07E1010EDBCFB0FEDC
:1070DA00020EDBCFB1FE50D0050EDF5C07E1010ED8
:1070EA00DBCFAEFE020EDBCFAFFE46D0080EDF5C72
:1070FA000FE12AEC41F0180ED880EE54000EED5440
:10710A0003E2180EF8EC3FF0010EDBCFAAFE34D0F2
:10711A00090EDF5C0FE12AEC41F0060ED880EE542E
:10712A00000EED5403E2060EF8EC3FF0010EDBCF41
:10713A00ABFE22D00A0EDF5C03E1FFEC3FF009D080
:10714A000B0EDF5C03E1FFEC3FF016D00C0EDF5CA8
:10715A0007E1010EDBCFB4FE020EDBCFB5FE0CD089
:10716A000D0EDF5C09E14BEC3FF004E00201010E79
:10717A00F36F02D00201F36B55EC2BF021EF41F0D3
:10718A00B6EC3EF0100EE12402E3E168E6520AECA6
:10719A0041F006EC41F0E66AD950040FCAEC40F01F
:1071AA0016EC40F0080FCAEC40F0E4EC3EF001E1C6
:1071BA00298C50EC40F002E629EC3FF005E2D95068
:1071CA00040F60EC3FF004D05CEC40F0B4EC3FF00C
:1071DA00A9EC3FF004E2600E4B6E9E0E52D068ECB2
:1071EA0040F002E62EEC3FF004E2320E4B6E9E0EA9
:1071FA0048D028EC40F09AEC3EF004E2020E4B6EC6
:10720A009E0E3FD086EC3EF00C0FEAEC3EF009E30E
:10721A0033EC40F00BEC3FF004E0DC0E4B6E9D0EBD
:10722A0030D074EC40F002E629EC3FF005E2D95088
:10723A00080F60EC3FF004D080EC40F0B4EC3FF073
:10724A0068EC40F002E62EEC3FF004E2AE0E4B6E24
:10725A009D0E17D028EC40F09AEC3EF004E27E0E28
:10726A004B6E9D0E0ED086EC3EF00C0FEAEC3EF013
:10727A000BE333EC40F00BEC3FF006E0580E4B6E9C
:10728A009D0ECEEC40F00BD0295009E13EEC40F0C7
:10729A0002E2E16AE552E16E4B5055EC2BF0100E1A
:1072AA00E15C02E2E16AE552E16EDEEF3EF0B6EC45
:1072BA003EF0180EE12402E3E168E6520AEC41F0DE
:1072CA00100EDB6A110EDB6A120EDB6A130EDB6A22
:1072DA00140EDB6A150EDB6A160EDB6A170EDB6A02
:1072EA0006EC41F0E66AD9500C0FCAEC40F0E66AA7
:1072FA00D950100FCAEC40F0E4EC3EF001E1298CC1
:10730A00100EDBCF4BF0110EDBCF4CF0120EDBCFA1
:10731A004DF0130EDBCF4EF0D9500C0F1AEC40F0A3
:10732A00EE504B26EE504C22EE504D22EE504E229D
:10733A00040E4BC0DBFF050E4CC0DBFF060E4DC032
:10734A00DBFF070E4EC0DBFF33EC40F0DBCF52F021
:10735A00D950100F1AEC40F0EE504F5C4B6EEE50C5
:10736A0050584C6EEE5051584D6EEE5052584E6E6B
:10737A00080E4BC0DBFF090E4CC0DBFF0A0E4DC0E6
:10738A00DBFF0B0E4EC0DBFF50EC40F002E629ECAF
:10739A003FF005E2D950040F6EEC3FF004D05CECEC
:1073AA0040F0C1EC3FF0A9EC3FF004E2600E4B6EF6
:1073BA009E0E4AD08CEC40F002E62EEC3FF004E23E
:1073CA00320E4B6E9E0E40D098EC40F004E2020E54
:1073DA004B6E9E0E39D086EC3EF0140FEAEC3EF06E
:1073EA0007E3A4EC40F004E0DC0E4B6E9D0E2CD0BB
:1073FA0074EC40F002E629EC3FF005E2D950080FA0
:10740A006EEC3FF004D080EC40F0C1EC3FF08CEC25
:10741A0040F002E62EEC3FF004E2AE0E4B6E9D0EFB
:10742A0013D098EC40F004E27E0E4B6E9D0E0CD009
:10743A0086EC3EF0140FEAEC3EF009E3A4EC40F0CF
:10744A0006E0580E4B6E9D0ECEEC40F00BD0295044
:10745A0009E13EEC40F002E2E16AE552E16E4B508E
:10746A0055EC2BF0180EE15C02E2E16AE552E16E9E
:10747A00DEEF3EF045EC41F0DE6A9DEC3FF01C5039
:10748A00FEE0D5EC40F08FEC3FF027E1B0EC40F0A5
:10749A0024E10201020E846FFA0EDBCF92F2FB0E98
:1074AA00DBCF93F2FC0EDBCF94F2FD0EDBCF95F22D
:1074BA00A3EC3FF092C23BF093C23CF094C23DF081
:1074CA0095C23EF0F1EC55F037C092F238C093F213
:1074DA0039C094F23AC095F2DFD00201926B936BF5
:1074EA00946B956B916B8D908B92D950F60F4FECF4
:1074FA003FF002E6DCEC3FF013E2020E9111916FCD
:10750A00E0EC40F003EC3FF0F60E37C0DBFFF70E7D
:10751A0038C0DBFFF80E39C0DBFFF90E3AC0DBFFDB
:10752A00D950F20F4FEC3FF002E6DCEC3FF014E2E8
:10753A00080E02019111916FEBEC40F003EC3FF061
:10754A00F20E37C0DBFFF30E38C0DBFFF40E39C092
:10755A00DBFFF50E3AC0DBFFD950F60F4FEC3FF0D8
:10756A0002E6E5EC3FF00BE2E0EC40F0DBCF3EF068
:10757A000F0E96EC3FF0FDE10FEC41F009D0D5EC8F
:10758A0040F02EEC41F096EC3FF0FDE1A3EC3FF029
:10759A0012EC3FF00CE2F4EC3EF0230E4B6E9D0E23
:1075AA00D0EC40F002E2E16AE552CEEC3FF0E4ECC6
:1075BA003EF012E1F60EDBCF4FF0F70EDBCF50F0C4
:1075CA00F80EDBCF51F0F90E0BEC3FF005E0F80EA8
:1075DA004B6E9C0E40EC41F0DFCF85F2010EDBCF03
:1075EA0086F2F60EDBCF89F2F70EDBCF8AF2F80EBF
:1075FA00DBCF8BF2F90EDBCF8CF2D950F20F4FECC6
:10760A003FF002E6E5EC3FF00BE2EBEC40F0DBCFBB
:10761A003EF00F0E96EC3FF0FDE10FEC41F011D079
:10762A00F20EDBCF4BF0F30EDBCF4CF0F40EDBCFD8
:10763A004DF0F50E2EEC41F096EC3FF0FDE1A3EC97
:10764A003FF0EBDB0BE2CBDBC30E4B6E9C0ED0ECB8
:10765A0040F002E2E16AE552CEEC3FF0B0DB08E12D
:10766A00B0EC40F005E0980E4B6E9C0E40EC41F0F9
:10767A00DFCF87F2010EDBCF88F2F20EDBCF8DF27D
:10768A00F30EDBCF8EF2F40EDBCF8FF2F50EDBCFEB
:10769A0090F20201010E846F1C6A040EE15C02E2A0
:1076AA00E16AE552E16E85D35CDB110EE12402E367
:1076BA00E168E65206EC40F0030EDB6A61DB100E6D
:1076CA00DB6A1C5003E10201840502E0000402E1C6
:1076DA00010EDF6E0201840523E1846B090E89C263
:1076EA00DBFF0A0E8AC2DBFF0B0E8BC2DBFF0C0E1E
:1076FA008CC2DBFF0D0E8DC2DBFF0E0E8EC2DBFFCE
:10770A000F0E8FC2DBFF100E90C2DBFF896B8A6BF4
:10771A008B6B8C6B8D6B8E6B8F6B906B010E1C6EF3
:10772A00000421E1006A010E05C0DBFF020E06C05B
:10773A00DBFF030E07C0DBFF040E08C0DBFF050EEC
:10774A0009C0DBFF060E0AC0DBFF070E0BC0DBFF1A
:10775A00080E0CC0DBFF056A066A076A086A096A2E
:10776A000A6A0B6A0C6AD950050FF9DAD950010F67
:10777A00F6DAD9500D0FF3DAD950090FF0DADFCF64
:10778A00E6FFE66A830E4B6E9C0EF1DA4E6E150E1C
:10779A00E15C02E2E16AE55208EC40F0110EE15CBC
:1077AA0002E2E16AE552E16E04D3ECC24BF04C6AA4
:1077BA004BBE4C680CEC40F07E0E4D6E9C0E59DBB5
:1077CA0002E2E16AE552E16E505055EF2BF0C6EC49
:1077DA0040F0DE6ADD6A010EE66E25EC41F0030E2A
:1077EA00B9DA29500EE10201EC0504E111EC40F08E
:1077FA00E66A04D011EC40F0010EE66EEADB55ECC5
:10780A002BF0E552E552D5D2C6EC40F07FDB010EF3
:10781A00F36E030EF3CFDBFF4BEC40F016EC40F0B7
:10782A00030F44DB4DEC41F0E76E040EE7CFDBFFBC
:10783A0029502AE1030EDB50070805E2010EF36E18
:10784A00030EF3CFDBFFDF50010802E2010EDF6E09
:10785A00030EDB50030F0E01B65D0BE048DB02E2BC
:10786A00E16AE552E16E4B50030EDB50030F0E0145
:10787A00B66F010EDBCFE6FF020EDBCFE6FFDFCFEE
:10788A00E6FFA7DB55EC2BF0050EE15C02E2E16AAC
:10789A00E552E16E8ED245EC41F0FD0EDB040BE1C0
:1078AA00B0CEDEFFB1CEDDFF020EB2CEDBFF030E9D
:1078BA00B3CEDBFF0AD0AECEDEFFAFCEDDFF020EC7
:1078CA00B4CEDBFF030EB5CEDBFFFB0EDBCFE6FF4C
:1078DA00FC0EDBCFE6FF020EDBCFE6FF030EDBCFAB
:1078EA00E6FFB6CEE6FF98DB05EC53F04B6E070ECB
:1078FA00E15C02E2E16AE552E16E4B50040EE15CA2
:10790A0002E2E16AE552E16E54D2C6EC40F0E65278
:10791A00CADAFFEC40F038E1295054E10201EB5198
:10792A0003E0020EEB5D28E1DF50000821E2EB5193
:10793A0001E18D90DF0403E18D848D82898C020E32
:10794A00DF5C03E18D848D82899C030EDF5C03E199
:10795A008D948D82899C040EDF5C03E18D848D9267
:10796A00899C050EDF5C10E18D948D92899C0CD068
:10797A00EB510AE18D8008D0EB0506E1DF500008E3
:10798A0002E28C9201D08C824CDB010F8FDAFFEC81
:10799A0040F016E1295016E10201EB5108E1010E0F
:1079AA00DB50000802E28B920BD08B8209D0EB05E8
:1079BA0007E1010EDB50000802E2899201D08982B8
:1079CA0055EC2BF021EF41F0FE0E0201ED5DFF0EAA
:1079DA00EE59FF0EEF59FF0EF05905E2ED2B000E9E
:1079EA00EE23EF23F02355EF2BF00201ED51EE11B8
:1079FA00EF11F01105E0ED07000EEE5BEF5BF05BB7
:107A0A0055EF2BF045EC41F0E65206EC41F0E76EFB
:107A1A00040EE7CFDBFFDB500BE1DFCFEDF2010E07
:107A2A00DBCFEEF2020EDBCFEFF2030EDBCFF0F28A
:107A3A0055EC2BF0050EE15C02E2E16AE552E16EDB
:107A4A00B8D1EDC2E6FFEEC2E6FFEFC2E6FFF0C232
:107A5A00E6FF750E4B6E9C0E9EDB02E2E16AE55272
:107A6A0008EF40F0E66AF10EE66E020EE66E4DECA5
:107A7A0041F0295001E0120055EF2BF0F1C24BF012
:107A8A004C6A4BBE4C68C3DA6E0E4D6E9C0EF1D931
:107A9A0002E2E16AE552E16E505055EF2BF0F2C274
:107AAA004BF04C6A4BBE4C68B2DA680E4D6E9C0EB7
:107ABA00E0D902E2E16AE552E16E50500201F26B4E
:107ACA0055EF2BF09DBCFED716C1E6FF17C1E6FFA6
:107ADA0000C1E6FF01C1E6FF5C0E4B6E9C0E5BDB4C
:107AEA0002E2E16AE55208EF40F03BD90FDACEDA5A
:107AFA00295064E1AADBFF0ED880EE54030EED5440
:107B0A0007E2010EDB68030EF36E020EF3CFDBFF12
:107B1A00DF50010802E2010EDF6EB8D907E1DF0487
:107B2A0005E10201F56B020EF66F06D0010EDBCFFE
:107B3A00F5F2020EDBCFF6F2CAB415D0CB68FC0E12
:107B4A00CA140009CA6E9D920F0152815293F00E17
:107B5A00BA140C09BA6E3F0EBA140009BA6E0E01B5
:107B6A000E0ECC6FCA84DF5023E0F5C24BF0F6C28A
:107B7A004CF0D8904C324B32D8904C324B324B505E
:107B8A00BB6EF5C24DF0F6C24EF0040ED8904D36DB
:107B9A004E36E804FBE1300E4D16000E4E16CF0E9F
:107BAA00BA1400014D104B6E4EC04CF0E85003D091
:107BBA00BB6ACF0EBA14BA6E55EC2BF03DD3120045
:107BCA00D0D81B0EE12402E3E168E6521ADAF29EEB
:107BDA00030E00C0DBFF040E01C0DBFF050E02C06E
:107BEA00DBFF060E03C0DBFF070E04C0DBFF080E37
:107BFA0005C0DBFF090E06C0DBFF0A0E07C0DBFF6C
:107C0A000B0E08C0DBFF0C0E09C0DBFF0D0E0AC00D
:107C1A00DBFF0E0E0BC0DBFF0F0E0CC0DBFF100EDE
:107C2A000DC0DBFF110E0EC0DBFF120E0FC0DBFF13
:107C3A00130E10C0DBFF140E11C0DBFF150E12C0AD
:107C4A00DBFF160E13C0DBFF170E14C0DBFF180E86
:107C5A0015C0DBFF190E16C0DBFF1A0E17C0DBFFBB
:107C6A00F28E110EDBCF4BF0120EDBCF4CF0130E5F
:107C7A00DBCF4DF0140E4ED902E0010EDF6E030E7B
:107C8A00DB5002E0010EDF6E1C5002E1010EDF6ED6
:107C9A00DF500FE0080EDBCF4BF0090EDBCF4CF0C4
:107CAA000A0EDBCF4DF00B0E35D903E0DE52010E82
:107CBA00DD6EDF5008E0C7D92DD905E0010EF36E5D
:107CCA00020EF3CFDBFF020EDBCFE6FFE66A010E00
:107CDA00DBCFE6FFE66ADFCFE6FFE66A4E0E4B6EC3
:107CEA009C0E45D84E6E090EE15C02E2E16AE5524D
:107CFA00E16E4E501B0EE15C02E2E16AE552E16E72
:107D0A0058D035DA1F0E406E050E416E426A436A3C
:107D1A0091D97CEC56F03BC04BF03CC04CF03DC0D6
:107D2A004DF03EC04EF0D9501200DBCF4EF082D952
:107D3A00DFCF40F0010EDBCF41F0020EDBCF42F085
:107D4A00030EDBCF43F07CEC56F0D880190E3B547F
:107D5A0014EF41F0E66E98EC30F0E55295D265D911
:107D6A0040D26EDAE1CFD9FFE2CFDAFF12004C6ED1
:107D7A004D6A4BC0E6FFE66E4DC0E6FF1BEF55F0BD
:107D8A00040EDB6A050EDB6A060EDB6A070EDB6A87
:107D9A00080EDB6A090EDB6A0A0EDB6A0B0EDB6A67
:107DAA000C0EDB6A0D0EDB6A0E0EDB6A0F0EDB6A47
:107DBA001200E552E5CFDAFFE7CFD9FF1200D7D993
:107DCA004B504C104D104E1012002FD9EE503B5C08
:107DDA00EE503C58EE503D58EE503E58120041DAF3
:107DEA0000D2FA0EDBCF40F0FB0EDBCF41F0FC0EE7
:107DFA00DBCF42F0FD0EDBCF43F01200DBCF3EF0CB
:107E0A004068416842684368F1EF55F0DBCF52F0B1
:107E1A004F5050105110521012007CEC56F03BC0DB
:107E2A00DEFF3CC0DEFF3DC0DEFF3EC0DDFFDD52AF
:107E3A00DD5217DAD880000EEE54800EEE54000E92
:107E4A00EE54000EEE541200D880E9D9000E3F54C9
:107E5A001200D880FF0E3C54FF0E3D54FF0E3E54D4
:107E6A00000E3F541200DBCF3FF03F34000E3F18A4
:107E7A0012004E6E4F6A4DC0E6FFE66E4FC0E6FF37
:107E8A001BEC55F0506E050EE15C1200DED9EE5087
:107E9A00ED101200E96EFF0EDA20EA6ED890030E9A
:107EAA00EB50000A1200E66A25EF41F0E66E000E7A
:107EBA00DA20E66E1200B9D80C0EEECFDBFF0D0EFB
:107ECA00EECFDBFF0E0EEECFDBFF0F0EEECFDBFFAA
:107EDA001200ABD8140EEECFDBFF150EEECFDBFF90
:107EEA00160EEECFDBFF170EEECFDBFF1200000EF1
:107EFA00E66EE66AE66EE66AB6CEE6FFE66EE66A23
:107F0A0005EC53F04B6E070EE15C1200E652E652A6
:107F1A00E6528CD1DBCF4EF04B504C104D104E1028
:107F2A001200D8903B363C363D363E36E806120003
:107F3A00DE6ADE6ADD6ADD52DD521200190E406E1B
:107F4A00416A426A436A12008CD9D880FF0EEE5405
:107F5A00FF0EEE54FF0EEE54000EEE5412000C0EFD
:107F6A0037C0DBFF0D0E38C0DBFF0E0E39C0DBFF5A
:107F7A000F0E3AC0DBFF1200140E37C0DBFF150EDE
:107F8A0038C0DBFF160E39C0DBFF170E3AC0DBFF25
:107F9A001200E16E4E50DE6A800EDE6EDE6ADD6A27
:107FAA00DD52DD52120051D9010EEE181200000EF8
:107FBA00EE5C000EEE58000EEE58000EEE5812005F
:107FCA00FF0EEE5CFF0EEE58010EEE58000EEE5854
:107FDA00120061DC59D1EB6F96809482958C958E54
:107FEA009588958A1200F36E010EF3CFDBFF020E1D
:107FFA00DB6A1200010EDBCFB2FE020EDBCFB3FE4C
:10800A001200E16E13D1E16E4E5055EF2BF04BC0CA
:10801A00E6FF4CC0E6FF1200DECFE6FFDDCFE6FF4B
:10802A001200010EE66ED9501200E96E000EDA2037
:10803A00EA6E12004BC03BF04CC03CF04DC03DF024
:10804A004EC03EF012000C0EDBCF4BF00D0EDBCF14
:10805A004CF00E0EDBCF4DF00F0E12000C0EDBCFE4
:10806A004FF00D0EDBCF50F00E0EDBCF51F00F0E9E
:10807A001200D950080F73DED950040F70DEAFDE3C
:10808A003FEC3AF04B6E0C0EE15C12000CDF00D9AB
:10809A00C8DF3BEF41F0040EDBCF3CF0050EDBCF2F
:1080AA003DF0060EDBCF3EF0070E38EF3FF0040E30
:1080BA00DBCF3BF0050EDBCF3CF0060EDBCF3DF00D
:1080CA00070E03EF3FF00C0EDBCF3CF00D0EDBCFBB
:1080DA003DF00E0EDBCF3EF00F0E38EF3FF0080EEC
:1080EA00DBCF3CF0090EDBCF3DF00A0EDBCF3EF0D2
:1080FA000B0E38EF3FF0080EDBCF3BF0090EDBCF5B
:10810A003CF00A0EDBCF3DF00B0E03EF3FF0140EEE
:10811A00DBCF3CF0150EDBCF3DF0160EDBCF3EF089
:10812A00170E38EF3FF0140EDBCF4BF0150EDBCFF6
:10813A004CF0160EDBCF4DF0170E9AEF3EF0140EF0
:10814A00DBCF4FF0150EDBCF50F0160EDBCF51F020
:10815A00170E0BEF3FF0F20EDBCF4FF0F30EDBCF33
:10816A0050F0F40EDBCF51F0F50E0BEF3FF079D85B
:10817A00EECF4BF0EECF4CF0EECF4DF0EFCF4EF00E
:10818A001200EFDDE652E652120090DE060EAFEF65
:10819A003EF0EDDD79D0EBDD4E6E070EE15C1200AC
:1081AA00F60EDBCF4BF0F70EDBCF4CF0F80EDBCF41
:1081BA004DF0F90E1200F60EDBCF3BF0F70EDBCFD7
:1081CA003CF0F80EDBCF3DF0F90E1200F20EDBCFD9
:1081DA003BF0F30EDBCF3CF0F40EDBCF3DF0F50EB7
:1081EA001200EECFE6FFEECFE6FFEECFE6FFEFCFCF
:1081FA00E6FF12004DD8E76E020EE7CFDBFFDB5039
:10820A00120051DE070EAFEF3EF0E16EDE6A90DE3D
:10821A00C5EF3EF093DE7CEC56F0F6EF3EF0000E32
:10822A003C54000E3D54000E3E541200DF6A010E0B
:10823A00DB6A020EDB6A1200E552E552E552B9D555
:10824A00D9CFE6FFDACFE6FF1200D950010F1AEFB5
:10825A0040F0DBCF4EF0EEDEC4DD7CEC56F00F0EC4
:10826A001200D9CFE9FFDACFEAFF1200010F1EDEB2
:10827A00030EAFEF3EF08DDF010EDE6E9DEF3FF095
:10828A0080DFE652E6521200E552E552E55212004C
:10829A00010EAFEF3EF0E7EC46F0A098636A626A1F
:1082AA000F01266BBEEC47F002E2E16AE552E16E8D
:1082BA004B500F017BEC47F0DF6ADF504B6E4C6A84
:1082CA000C0E4B5C000E4C5810E2DF50040DF3CF3D
:1082DA00E9FFF4CFEAFF000EE926040EEA22EE6A6D
:1082EA00EE6AEE6AEE6ADF2AE8D7658C0F01386B10
:1082FA006598659C62A607D062960601BF6BC46B3F
:10830A00C56BC66BF7D70601010ED86FD96FDA6B4A
:10831A00DB6BCC6BDF6A030EDF5C11E2EA6ADF34E7
:10832A00EBEC47F0EA22EE6AED6AEA6ADF34F2EC35
:10833A0047F0EA22EE6AED6A25EC47F0ECD706012F
:10834A00080EB56F040EB66F0F01160E266F0401E4
:10835A00300E026F040E036F400E016F840E006F21
:10836A000601A96BA86BEAEF46F0E7EC46F082BE7D
:10837A0006D0656A0F01366B0601A86B7CD0060130
:10838A00A8510CE1656A0F01366B7BEC47F065B6C4
:10839A0002D06586FCD70601010EA86FA8050AE17E
:1083AA0065BA08D0626A0F01366B368136890601D2
:1083BA00020EA86F6250040B06E00F013651040B3F
:1083CA0002E062943EDB65B256D06250010B09E0CE
:1083DA000F013651010B05E05EDF0601040EA86F9E
:1083EA0062906250100B06E00F013651100B02E04A
:1083FA0018DB629862AC15D00F0136AD0AD082EC58
:10840A0047F0730EF1EC46F002E2E16AE552E16EE2
:10841A004B50629C0601D65101E0D607D65101E1C4
:10842A00F3D86250200B05E00F013651200B01E012
:10843A00E7DA6250020B14E00F013651020B10E02A
:10844A0082EC47F0E6687F0EE66E2CEC54F04B6E39
:10845A00060EE15C02E2E16AE552E16E4B50636AA4
:10846A00040E0601E76EA819E8AE02D0E73402D07E
:10847A00E750A85D02E2A19834D00F0136A730D0A8
:10848A00DF6A040EDF5C2CE262A62AD064CFCDF646
:10849A000601CD51780BE842E842E842CE6F629677
:1084AA00CDB504D0CE51F9EC47F003D0CE51FEEC55
:1084BA0047F0EA22EF70CE5102E1D5DA0FD0000E72
:1084CA00E66EE66ACD0EE66E060EE66E720EF1EC0A
:1084DA0046F002E2E16AE552E16E4B50DF2AD1D75B
:1084EA00A198EAEF46F0E8EC47F0FC0EDBA403D0D3
:1084FA00E66A63EC47F0FC0EDBA204D0010EE66EDE
:10850A0063EC47F0FD0EDB504C6A260F4B6E0F0EE4
:10851A005DEC47F0F9EC46F0FC0EDBCFEFFFE552DD
:10852A00EAEF46F0E8EC47F0FC0EDB5003E0ECEC37
:10853A0046F002D016EC47F049EC47F0D9CFE9FFF4
:10854A00DACFEAFFEE50ED1003E1F36AF46A28D0BD
:10855A00F9EC46F00DEC48F0FA0EDBCFEEFFFB0E1D
:10856A00DBCFEDFFF9EC46F0EE52F90EDBCFEFFF71
:10857A00400E03EC48F0880E12EC48F0FC0EDB507B
:10858A0003E0ECEC46F002D016EC47F0EA22EF7476
:10859A00DECF4BF0DDCF4CF04BC0F3FF4CC0F4FF05
:1085AA00E552EAEF46F0E8EC47F0FD0EDB5003E156
:1085BA00C7EC47F009D01BEC47F09CEC47F01BECEA
:1085CA0047F0010F9CEC47F0E552EAEF46F0CEEC9B
:1085DA0047F065A817D0E1EC47F0400EEE16EE6AB8
:1085EA00EE6AEE6AE1EC47F0EE7CECEC46F0EA2249
:1085FA00EF74400E4B6EE1EC47F04B50EF16E1EC96
:10860A0047F0EF7CB8EF47F00601D85123E1010E9D
:10861A00D86FD9511FE1010ED96F020EBC5D07E177
:10862A00E8DBEE52EF6AE5DBC80EEF6E1200BC051E
:10863A0011E1CF6B0BEC47F0EE52400EEF6EE6DB2A
:10864A00A8EC47F0E3DB840EEF6E010ECF6FB6DBCA
:10865A00800EEF6E12000601DA6BDB6B020EBC5D58
:10866A0006E107EC48F0D7DB97EC47F010D0C05191
:10867A000401365D0601C1510401375904E236C4CA
:10868A00C0F637C4C1F65CD8B4DBC5DBB2DBC80EB2
:10869A00EF6E1200E8EC47F0000EDE6E040EDD6E9F
:1086AA00C5DB040DF4CF4CF0D9CFE9FFDACFEAFFEE
:1086BA00F350EE264C50ED2297DBEF9EFC0EDB507A
:1086CA0002E1AFDB01D083DBEA22DECFEEFFDDCFB2
:1086DA00EDFF8ADBEF9C88DB040EE926000EEA2216
:1086EA00EF8CE55272D365980601BFBF0DD0C4AFB7
:1086FA0009D0020EBC6FDB5101E1ADDF0601D96B77
:10870A00D86B1200C7EF47F0040130AF0DD0060155
:10871A00010EBC6FDA5101E19EDF0601D96BD86BFD
:10872A00D7510DE109EF43F00601020EBC6F46DB9B
:10873A00840EEF6ED96BD86BD75101E165DF120059
:10874A0041DB400EDF6E0601C05D000EC1590AE230
:10875A00C0C6DFFFBB5102E1010E03D0BB0502E137
:10876A00020EBB6FDF504C6AE850C05DC06F4C50C0
:10877A00C159C16F3EDBEE52DFCFEFFF380EC96F32
:10878A00040ECA6FBFB10DD0DF5017E0BDC6F6FFA9
:10879A00BEC6F7FFBD2B000EBE230800F55067DBEF
:1087AA00F3D7DF500AE0BDC6E9FFBEC6EAFFBD2B1C
:1087BA00000EBE23EF505BDBF4D707D3E8EC47F09B
:1087CA0025DBEE52EFCFDFFFDFCF4BF04B50060138
:1087DA00C55D000EC65902E2C5C6DFFFDF504B6E0B
:1087EA004C6AE850C55DC56F4C50C659C66F010E3C
:1087FA00DB6ADF50F36E010EDBCFF4FFF350F45C5B
:10880A0016E2010EDB50EA6A380FE96E040EEA221C
:10881A00EF50E66EC2C6E9FFC3C6EAFFC22B000EDE
:10882A00C323E552E750EF6E010EDB2AE2D7000EB2
:10883A00D880C555000EC6550DE2E4DBECDAE6DA5F
:10884A00EF50400B03E16EDBC80E02D06BDB880EE3
:10885A00EF6E12D0B3DA840EEF6EC751C81107E07B
:10886A0005D0C8C6FAFF0601C751F96EFADF06013C
:10887A00C49FD75101E1C8DEE552A7D2A3DA0601A7
:10888A00BF8F77DB02E2E16AE552E16E4B50300EB0
:10889A00E66EE66AE66A000EE66E040EDBDA02E2CD
:1088AA00E16AE552E16E4B50658CDF6A030EDF5CCC
:1088BA0002E2C6DAFBD7010EE66EE66AE66AAA0E9D
:1088CA00E66E060EC7DA02E2E16AE552E16E4B5045
:1088DA00659C0601080EB56F040EB66F000EAB6FED
:1088EA00040EAC6FABC6ADF6AE6F32C4A9F6A95191
:1088FA0002E1100E10D0010EE66EE66AA90EE66ECF
:10890A00060EE66E010E68DA02E2E16AE552E16EEF
:10891A004B500601200EA86F58D2800E0401305D1C
:10892A0038E10601C00EBF6F04013351030A1AE091
:10893A00010A09E0030A2BE10601CE0EBD6FAA0E59
:10894A00BE6F120E1ED0E7DA550EF626AB0EBEDA51
:10895A00020E0601D9DAF5CFC0F6030ED5DAF5CF45
:10896A00C1F61200030E325D0FE2D5DA570EF62673
:10897A00AB0EACDABDC6F6FFBEC6F7FF0800F5506F
:10898A000601C06FC16B12000601BF6B120006011F
:10899A00BF6B120018DB0401386B396B30511F0BA7
:1089AA00020A11E0030A0CE0010A1EE10601BF8F68
:1089BA00040138810601CB0517E10401388314D07C
:1089CA000601BF8F11D00601BF8F040134BF02D048
:1089DA00E9DA01D0ECDA58DAF2DA06E005DAEF5031
:1089EA00040B02E0010E386F0601BFAF07D0380E44
:1089FA00BD6F040EBE6FBF81020EC06FE552E5D196
:108A0A000F0126A10CD002DAEF50800807E1F1D954
:108A1A00EF50840803E1FAD98C0EEF6E2691629A20
:108A2A0012000F013685629865820601010ECC6F2D
:108A3A0031DA750ED1D902E2E16AE552E16E4B50A4
:108A4A0012000601CC6B26DA740EC6D902E2E16A7C
:108A5A00E552E16E4B5065920F01369562A402D041
:108A6A006294FCD71200AED906012D0ED66FFD0E08
:108A7A00CD1539E17E0ECD15E8407F0B040DF3CFFD
:108A8A00ABF6F4CFACF6000EAB27040EAC23ABC6A4
:108A9A00ADF6ACC6AEF6AD75B9D9EF503C0BE842AF
:108AAA00E8420D081EE1DF6A080EDF5C16E2AED965
:108ABA00020EE926000ED5D9EF50E66EDF50EA6ABB
:108ACA00300FE96E040EEA22E552E750EF6E9ED9A6
:108ADA009FDAEE2AEF22DF2AE7D798D934DA09D8C3
:108AEA0007D027D805D0FD0ECD15040801E130D8EE
:108AFA006CD10601BB6BD76BDA6BDB6BCF6BBC6BD4
:108B0A0078D9EF9EB57575D9EF9EB5750BDAEF9EDC
:108B1A00BF6BC06BC16BC46BC56BC66B55D8BAD97A
:108B2A00030E5AD902E2E16AE552E16E4B5078EF40
:108B3A0043F0020E0601BC5D02E1E3EF43F0BC6BB9
:108B4A00CF5104E13BD98C0EEF6E1200CF6B1200AD
:108B5A0039D94FD9EF50400B01E0010EDF6E060103
:108B6A00B575080EA85D0BE132C438FF0F01385104
:108B7A0003E00601100E02D00601040EA86FBC0520
:108B8A0013E137D948D9DCDD020E0601BB5D03E1EA
:108B9A0030D9840E07D0DF5003E12BD9C80E02D09A
:108BAA0028D9880EEF6E0FD0C4AF0CD0C751C811A8
:108BBA0007E005D0C8C6FAFF0601C751F96EFADF09
:108BCA000601C49FBC6B01D104013051600BE8421D
:108BDA00E842E842E842E842000901E01200315165
:108BEA000C0A4AE00B0A3FE00C0A31E0010A22E0D3
:108BFA000B0A1EE0020A1CE0030A18E0080A10E049
:108C0A00010A0CE00F0A08E0030A01E0120006015B
:108C1A00BF8F080EA86F120092EF44F043EF44F0A2
:108C2A000601A90EBD6F060EBE6F0CD0CFEF44F041
:108C3A0042EF46F034510601BD6FBE6BAA0EBD2746
:108C4A00060EBE23BF81010EC06FBF8F1200060140
:108C5A00BF8F04013451EA6AAA0FE96E060EEA22AE
:108C6A0032C4EFFF120016D9020EB6D802E2E16A48
:108C7A00E552E16E4B5012001200A5D9E652E652B7
:108C8A00E6520401320510E130511F0B00090CE1D4
:108C9A000601BF8F030E0401315D04E10601010ED6
:108CAA00CB6F02D00601CB6B0401325101E07FD0B9
:108CBA0030511F0B020801E07AD034510F0B000922
:108CCA0001E175D034510F0B020871E3200E060141
:108CDA00A85D6DE1BF8F040134BF04D063D9D4D835
:108CEA00DFD803D064D9D0D8DFD8EA22020EEFCF7A
:108CFA00DBFFF4D8010B02E1DF9401D0DF8434BF3B
:108D0A0002D050D901D053D9EA22DECFEEFFDDCF0F
:108D1A00EDFF030E315D0CE152D907E034BF02D0FA
:108D2A00BFD801D0C1D8EA22EF82840E76D93FD0CB
:108D3A00DF7445D90BE058D8EF9E56D8EF8C09D985
:108D4A0002E2E16AE552E16E4B5002D04DD8EF8C57
:108D5A00DF74C4D8020B02E132D912E0040134BF35
:108D6A0002D09ED801D0A0D8EA22EF923B0E4B6ED9
:108D7A0045D9EFD802E2E16AE552E16E4B5002D0E2
:108D8A003B0E3CD9040134510F0B4C6A260F4B6E33
:108D9A000F0E4C22030E4BC0DBFF040E4CC0DBFF50
:108DAA00030EDBCFE9FF040EDBCFEAFFEF90050EDF
:108DBA00E15C02E2E16AE552E16ED5D023D9C3D87B
:108DCA0097EF47F0E6D8E6521200E552CCD0FD0EF6
:108DDA00EA6ADB34EBEF47F0E66EE66A2CEC54F015
:108DEA004B6E060EE15C1200DECFE9FFDDCFEAFF33
:108DFA001200B5C6E9FFB6C6EAFF120034510F0BDE
:108E0A00E96EEA6AD890E936EA361200ABC6E9FF9B
:108E1A00ACC6EAFF1200FCD8380EEE6E040EED6EF8
:108E2A001200FD0EEA6ADB34F2EF47F0FC0EDB506B
:108E3A00E8244D6EFD0EDB50040DF3504D24120054
:108E4A00DF50D7D8EA22EF6ADF50CED8EA22EF6A9B
:108E5A00DF2A1200E66ECEEC54F04B6E050EE15C92
:108E6A001200EA22EE50EFCFEAFFE96E1200E66E38
:108E7A00C9C6E9FFCAC6EAFFC92B000ECA23E552D2
:108E8A00E750EF6EDF061200EA22EECFDEFFEDCFEB
:108E9A00DDFF1200000EE66EE66AE66EE66A120072
:108EAA0034510F0BF9EF47F034510F0BFEEF47F037
:108EBA004C224BC0DEFF4CC0DDFF1200FD0EDBCFA3
:108ECA00E6FF4FEC43F0E552E5521200F7220900A3
:108EDA00F5CFBDF60A00F5CFBEF61200D950020F43
:108EEA00E96E000EDA20EA6EEF501200160E396FA4
:108EFA009F0E376F7B0E366F1200010EE66EE66A22
:108F0A00000EE66EE66A1200F76ABD25F66EBE51DD
:108F1A00F722080012003251F66EF76AD890F63638
:108F2A00F7361200ADC6E9FFAEC6EAFF1200040D1D
:108F3A00F3CF4BF0F4CF4CF0000E4B26040EB8DF03
:108F4A00840E12EF48F064D8300EEE6E040EED6E09
:108F5A001200020EE66EE66ADECFE6FFDDCFE6FF1E
:108F6A00050EF1EF46F0E552E5CFDAFFE7CFD9FF7C
:108F7A001200020EE66EE66AE66A270EE66E0F0E2B
:108F8A002FEF47F01BDF8C0EEF6E33DF840EEF6E90
:108F9A001200D9CFE6FFDACFE6FFE1CFD9FFE2CF61
:108FAA00DAFF12002BDFAF0EE926060E120026DFCB
:108FBA00B50EE926060E12000ADF36EF47F014DF77
:108FCA00EF50800B1200FEDEE6521200FE0BEA366C
:108FDA00E96EB50EE926060E1200FE0BEA36E96EB8
:108FEA00AF0EE926060E1200EA6AD30FE96E060EE4
:108FFA001200EA6AD00FE96E060E1200F5DEE8509A
:10900A00EF1612008FDFEE52400EEF6E97EF47F029
:10901A00020EE926000EEA221200E6DEE850EF12FE
:10902A00120052EC4DF0FB0EDBCFF3FFDB06F350E0
:10903A0000090AE0A0EC4DF0FA0E0BEC4EF0F3E159
:10904A004C1CF1E1010E01D0000E81EF4DF052EC03
:10905A004DF03B0EE12402E3E168E652E16E010EB7
:10906A00DB6A020EDB6AF90EDBCFF6FFFA0EDBCF04
:10907A00F7FFFB0EDBCFF8FF0800F550DF6EDF507D
:10908A0002E1A5EF4CF0250EDF5C02E098EF4CF010
:10909A00030EDB6A040EDB6A050EDB6A060EDB6A68
:1090AA00070EDB6ABAEC4CF02D0EDF5C0CE02B0EDF
:1090BA00DF5C09E0200EDF5C06E0230EDF5C03E0E4
:1090CA00300EDF5C1AE1DF50300A14E0130A0FE0B9
:1090DA00030A0AE00B0A05E0060AE4E1030EDB8054
:1090EA00E1D7030EDB82DED7030EDB84DBD7030E68
:1090FA00DB86D8D7030EDB88D5D72A0EDF5C1BE1C7
:10910A00B6EC4CF004EC4DF010E0030EDB803D6849
:10911A003E68130EDBCF42F0140EDBCF43F029EC8E
:10912A0056F0040E3BC0DBFF03D0130EEDEC4CF0FF
:10913A00BAEC4CF00BD0090EDB6A5BEC4DF003E0A5
:10914A00CFEC4DF0FAD7090EEDEC4CF0030EDBB084
:10915A00DB982E0EDF5C1BE1BAEC4CF02A0EDF5CCA
:10916A000BE1B6EC4CF004EC4DF003E1130E3FECCE
:10917A004DF0BAEC4CF00BD0090EDB6A5BEC4DF00B
:10918A0003E0CFEC4DF0FAD7090E3FEC4DF0680E34
:10919A00DF5C07E1BAEC4CF0680EDF5C1DE1030E00
:1091AA0018D0740EDF5C17E07A0EDF5C14E0480E0C
:1091BA00DF5C06E0540EDF5C03E05A0EDF5C02E17E
:1091CA00020E07D06C0EDF5C03E06A0EDF5C04E17E
:1091DA00010E92EC4DF0C9DBDF506E0A01E17FD33C
:1091EA001E0A01E192D1200A01E18FD13F0A01E171
:1091FA0049D11A0A01E146D10D0A01E143D1200AF7
:10920A0001E140D13A0A01E13DD1200A01E13AD116
:10921A00260A01E135D10D0A01E132D11A0A01E12A
:10922A00D9D0200A4AE0300A1FE0460A0EE0250A91
:10923A0001E083D3D950F90FE96EFF0EDA20EA6E06
:10924A00010EEE5E000EEE5AEE5AA0EC4DF0250E1F
:10925A00E66E95DB03E14C1C01E169D39CEC4DF011
:10926A0001E26BD3DB2A69D3080EDB6A040EDB50FA
:10927A00010806E2040EDB0464EC4DF0DB508BDBE4
:10928A00080EDB5009E0030EDB50010B05E172DB2F
:10929A0001E04DD3080EDB6A64DBEFCFDFFF14EC8D
:1092AA004EF003E14C1C01E142D39CEC4DF001E38A
:1092BA00DB2A60DB01E141D33AD3070EDB50020817
:1092CA000FE1E0EC4DF0030EA7EC4DF00E0EEECFE1
:1092DA00DBFF0F0EEECFDBFF100EEECFDBFF20D051
:1092EA00F70EDBCF4EF0F80EDBCF4FF0020E4E5EDC
:1092FA00000E4F5AF70E4EC0DBFFF80E4FC0DBFFD1
:10930A004EC0E9FF4FC0EAFF97EC4DF04D6A0E0ED2
:10931A004BC0DBFF0F0E4CC0DBFF100E4DC0DBFF56
:10932A000E0EDBCFE6FF0F0EDBCFE6FF100EDBCF14
:10933A00E6FFF6EC54F0E552E552E552130E3CC056
:10934A00DBFF140E3DC0DBFF060EDB5005E0130EFB
:10935A00DBEC4DF001E26ADBFFEC4DF002E2130EAA
:10936A0037DBC2EC4DF006E0040EDBEC4DF002E216
:10937A00050E2EDB030EDBB005D0FCDA01E0D7D2F6
:10938A00080EDB6A090EDB6A0E0EDBCFF6FF0F0E44
:10939A00DBCFF7FF100EDBCFF8FF0800F550DF6ECA
:1093AA00DF5014E005EC4EF011E214EC4EF003E14C
:1093BA004C1C01E1BCD2BBDB01E3DB2A090EDB2A30
:1093CA00D9500E0FE96E000ECBDBE7D7D3DA01E1F5
:1093DA00B4D2ADD2C6DA110EEECFDBFF120EEDCF4C
:1093EA00DBFF110EDBCFE6FF120EDBCFE6FFE8EC68
:1093FA0054F0E552E552130EF3CFDBFF140EF4CF0F
:10940A00DBFF060EDB5004E0130ED0DB01E20EDBBD
:10941A00FFEC4DF002E2130EDBDAAFDB05E0040EDF
:10942A00C5DB02E2050ED4DA030EDBB005D0A2DA00
:10943A0001E07DD2080EDB6A090EDB6A110EDBCF72
:10944A00E9FF120EDBCFEAFFEFCFDFFFDF5014E0B8
:10945A00D7DB12E2E4DB03E14C1C01E168D267DBF3
:10946A0001E3DB2A090EDB2A110EDB2ADBCFE9FF37
:10947A00120EE8E3DB2AE6D77DDA01E15ED257D2A3
:10948A00030EDB8E070EDB0410E195DB040E5ADBBC
:10949A000A0EEECFDBFF0B0EEECFDBFF0C0EEECF8C
:1094AA00DBFF0D0EEECFDBFF6CD0070EDB5003089F
:1094BA002CE1030EDBAE0DD0B2DA020E76DAEFCF74
:1094CA004BF04C6A4D6A4E6A4BAE39D04C684D68C7
:1094DA0035D0F70EDBCF4CF0F80EDBCF4DF0020E95
:1094EA004C5E000E4D5AF70E4CC0DBFFF80E4DC015
:1094FA00DBFF4CC0E9FF4DC0EAFFEFCF4BF00A0E8D
:10950A004BC0DBFF0B0EDB6A38D0070EDB500208BC
:10951A0009E1030EDBAE04D059DB4DAE10D00ED0FC
:10952A0055DB0DD0030EDBAE12D079DA020E3DDA2E
:10953A00F9DA4D6A4E6A4CAE02D04D684E68E2DAEC
:10954A000C0E4DC0DBFF0D0E4EC0DBFF1AD0F70E1E
:10955A00DBCF4DF0F80EDBCF4EF0020E4D5E000E63
:10956A004E5AF70E4DC0DBFFF80E4EC0DBFF4DC062
:10957A00E9FF4EC0EAFFD6DAC5DA0C0EDB6A0D0E39
:10958A00DB6A060EDB5005E1010EF36E050EF3CF22
:10959A00DBFF150EDB6A160EDB6AD950370F4B6EEE
:1095AA00000EDA204C6E390E4BC0DBFF3A0E4CC06F
:1095BA00DBFF380EDB6A080EDB6A0A0EAEDADF5012
:1095CA00780A12E0200A10E0280A0CE0200A0AE0D1
:1095DA003F0A06E00D0A02E0200A08E1020E05D061
:1095EA00080E03D0080EDF26100E97DA030EDBBE34
:1095FA0002D0DB92DB94DB50800B24E08ADAD8902D
:10960A00030EEB50000A08E6000EEE5C000EEE5860
:10961A00000EEE58000EEE5815E213DA4068416863
:10962A0042684368F1EC55F00A0E37C0DBFF0B0EB7
:10963A0038C0DBFF0C0E39C0DBFF0D0E3AC0DBFF72
:10964A002D0E08D0030EDBA202D02B0E03D0DBA412
:10965A0008D0200EF36E170EF3CFDBFF150EDB2AB0
:10966A0002D0170EDB6A050EDB5003E1B7D901E120
:10967A0089D0E40E4B6EAD0E4C6E000E4D6E070E89
:10968A00DBCF4EF04F6A506A516A4EC040F04FC06D
:10969A0041F050C042F051C043F0D3D97CEC56F0AF
:1096AA004B503724F36E4C503820F46E4D5039200D
:1096BA00F86EF4CFF7FFF3CFF6FF0800090EF5CFE7
:1096CA00DBFF580EDF5C0FE1610EF36E090E7BD9EA
:1096DA000AE3200E4B6E090EDBCFE7FF4B50E75E25
:1096EA00090EE7CFDBFF070EDBCF4BF04C6A4D6A62
:1096FA004E6A0FDA4BC040F04CC041F04DC042F008
:10970A004EC043F0EECF3BF0EECF3CF0EECF3DF053
:10971A00EFCF3EF07CEC56F03EC0EDFF3DC0EDFFD2
:10972A003CC0EDFF3BC0EFFF390EDBCFE9FFDB06A4
:10973A003A0EDBCFEAFF01E2DB06090EDBCFEFFFD1
:10974A00150EDB2A4BD995E1030EDBA61DD06F0E51
:10975A00DF5C06E1C1D918E3150EDB285BDA14D009
:10976A00780EDF5C09E0580EDF5C06E0620EDF5C13
:10977A0003E0420EDF5C08E1020EF36E160EF3CF31
:10978A00DBFF02D0150EDB6A030EDB50100B0EE076
:10979A00040EDBCF4BF0050EDB50D8804B5406E2AB
:1097AA00060EDB5003E1040EDB5034DA95D90AE2E7
:1097BA00050EDBCFE7FF150EDB50E75E050EE7CFA0
:1097CA00DBFF02D0050EDB6A040EDBCF4BF0160E70
:1097DA0045D9D8804B5414E2160EDBCFE6FF150E9E
:1097EA00DBCFE6FF040EDBCFE6FF050EDB50E552CA
:1097FA00E75CE552D880E754E552D880E7545FD950
:10980A00030EDB50010B0BE1080EDB5008E0B2D867
:10981A0001E08DD0080EDB50BED8080EDB6A170EA9
:10982A00DB5007E088D9170EF1D903E14C1C01E19E
:10983A007ED0160EDB5016E07ED9300EE66E9FD82B
:10984A0002E14C1C74E077D9DFCFE6FFAFEC55F0AC
:10985A00E552E552E552F4CF4CF00001F31C02E167
:10986A004C1C65E0050EDBCF4BF0160EDB50D880A2
:10987A004B5409E2050EDBCFE7FF160EDB50E75E1D
:10988A00050EE7CFDBFF300EE66E050ECBD94FE1B2
:10989A00390EDB2ADBCFE9FF3A0E01E3DB2ADBCF05
:1098AA00EAFF090EEFCFDBFFDB500EE044D9090EC9
:1098BA00ADD902E14C1C3BE0390EDB2ADBCFE9FFD4
:1098CA003A0EEDE3DB2AEBD755D831E1160EDBCFA2
:1098DA00E6FF080EC3D8E552E7245DD82ED0070E5E
:1098EA00DB50030A1CE0010A14E0030A07E07BD9F3
:1098FA00DBCFEEFF020EDBCFEDFF1FD0F5D8506AAB
:10990A004EAE02D04F6850682CD8BCD850C0EEFF7B
:10991A0014D0EAD84EBE4F6824D8B4D80ED063D932
:10992A00DBCFEFFF0AD07BD905E14C1C03E1F368DA
:10993A00F46810D0FCD801E3DB2A79D941EF48F06A
:10994A00010EDBCF4BF0020EDBCF4CF04BC0F3FF26
:10995A004CC0F4FF3B0EE15C02E2E16AE552E16EC3
:10996A00CBD029D9020EA7EF4DF061D90800F550E6
:10997A00DF6E1200200EE66E080E17EF4EF0AFEC07
:10998A0055F0E552E552E552F3CF4BF0F4CF4CF0E7
:10999A000001F31C12004B6E4C6AD950010F4DD9CD
:1099AA004B50EE264C50ED2212004F5E000E505ADC
:1099BA00F70E4FC0DBFFF80E50C0DBFF4FC0E9FFC8
:1099CA0050C0EAFF1200DBCFF4FFF350F45C120040
:1099DA00DB50E76E040EE7CFDBFF12000A0EDBCF87
:1099EA004BF00B0EDBCF4CF00C0EDBCF4DF00D0E17
:1099FA00DBCF4EF04B504C104D104E101200130E90
:109A0A00EECFDBFF140EEDCFDBFF130EDBCF4BF0F7
:109A1A00140EDBCF4CF00001800E4C141200F70E2E
:109A2A00DBCF4FF0F80EDBCF50F01200050EDB5003
:109A3A00E66ED950130F01D9E552E750EE6EED6A82
:109A4A0012000A0EDBCF3BF00B0EDBCF3CF00C0E04
:109A5A00DBCF3DF00D0EDBCF3EF01200DBCFE6FF91
:109A6A00150EDBCFE6FF050EDB50E552E724E55283
:109A7A00E7241200DB50CED8010EF36E060EF3CFA8
:109A8A00DBFF1200EE50EFCFEAFFE96E4DC0EEFFAA
:109A9A004EC0EEFF4FC0EEFF1200D9CFE6FFDACF7D
:109AAA00E6FFE1CFD9FFE2CFDAFF1200DFCFE6FF10
:109ABA00E66A6AEC56F0E552E552F3501200E76E98
:109ACA00080EE7CFDBFF1200EECF4BF0EECF4CF0E3
:109ADA00EFCF4DF04E6A1200050EDBCF4BF0150E9C
:109AEA00DB50D8804B541200010EDBCF4DF0020E32
:109AFA00DBCF4EF04F6A1200E552E5CFDAFFE7CF2F
:109B0A00D9FF12000A0E4BC0DBFF0B0E4CC0DBFF65
:109B1A001200D9500A0F22EF4EF0F36E070EF3CF60
:109B2A00DBFF1200EECF4BF0EFCF4CF01200010E2C
:109B3A00DB2A020E1200FC0EDBCFE6FFFD0EDBCFA6
:109B4A00E6FF12004B5E000E4C5AF70E4BC0DBFFCD
:109B5A00F80E4CC0DBFF4BC0E9FF4CC0EAFF120015
:109B6A00DA20EA6EEF2AEECFF6FF000EEF22EECFF2
:109B7A00F7FFEF22EECFF8FF1200040EDBCFE6FF6D
:109B8A00130EDB50E552E75C9ADFDB5004DF060E6A
:109B9A00DB501200090EDB500A0DF350DF24D00F00
:109BAA00E76E090EE7CFDBFFBAEF4CF0DB50F36E3E
:109BBA00050EE8EF4CF0F70EDBCF4BF0F80EDBCFDB
:109BCA004CF01200DFCFE6FFC4EF4CF028DF030EA3
:109BDA00ECDE69EF4DF016EC48F0E552E552E5523D
:109BEA00E55200091200BDDEEE50EFCFEAFFE96E42
:109BFA00010E1200130EDB50F36E040EE8EF4CF068
:109C0A00040EDB50F36E090EE8EF4CF0DBCFE6FFF3
:109C1A00C4EF4CF0E76E050EE7CFDBFF12008BDFD7
:109C2A00E7EF4DF0DBCFE6FF86DFF0EF4DF0D950DE
:109C3A00F90FE96EFF0EB5EF4DF0E96E000EDA206E
:109C4A00EA6E1200514D2C25692C25692C25690ACA
:109C5A000D00253034692C253034690D0A00253170
:109C6A00690D0A00253033690D0A00253031306C40
:109C7A00750D0A0025640A0D0025642C256C752CC7
:109C8A00256C752C256C752C256C750A0D004D619B
:109C9A006A6F72206D616C66756E6374696F6E208F
:109CAA0041786973322053746570436F756E7465B9
:109CBA0072207A65726F0A0D004D616A6F72206DAB
:109CCA00616C66756E6374696F6E20417869733270
:109CDA002053746570436F756E74657220746F6F6C
:109CEA002068696768203A20256C750A0D004D6165
:109CFA006A6F72206D616C66756E6374696F6E202F
:109D0A0041786973312053746570436F756E746559
:109D1A0072207A65726F0A0D004D616A6F72206D4A
:109D2A00616C66756E6374696F6E20417869733110
:109D3A002053746570436F756E74657220746F6F0B
:109D4A002068696768203A20256C750A0D00213061
:109D5A00204572723A203C61786973323E207374EE
:109D6A0065702072617465203C20312E3331487A47
:109D7A002E0A0D002130204572723A203C61786922
:109D8A0073323E20737465702072617465203E20C0
:109D9A0032354B2073746570732F7365636F6E640D
:109DAA002E0A0D002130204572723A203C617869F2
:109DBA0073323E206C6172676572207468616E202E
:109DCA0031363737373231352073746570732E0A5E
:109DDA000D002130204572723A203C617869733156
:109DEA003E20737465702072617465203C20312EA8
:109DFA003331487A2E0A0D002130204572723A20FA
:109E0A003C61786973313E207374657020726174A5
:109E1A0065203E2032354B2073746570732F73654D
:109E2A00636F6E642E0A0D002130204572723A204B
:109E3A003C61786973313E206C6172676572207487
:109E4A0068616E20313637373732313520737465A1
:109E5A0070732E0A0D002130204572723A203C6D33
:109E6A006F76655F6475726174696F6E3E206C61AE
:109E7A0072676572207468616E20313637373732FF
:109E8A003135206D732E0A0D005374617475733D5C
:109E9A0025690D0A002135204572723A204E656502
:109EAA006420636F6D6D61206E6578742C20666F17
:109EBA00756E643A20272563270D0A005061726186
:109ECA006D383D25630D0A00506172616D373D257D
:109EDA00630D0A00506172616D363D256C750D0A7D
:109EEA0000506172616D353D256C640D0A00506148
:109EFA0072616D343D25750D0A00506172616D33D2
:109F0A003D25640D0A00506172616D323D25640D74
:109F1A000A00506172616D313D25640D0A00504995
:109F2A002C2531750D0A004D522C253033750D0A3A
:109F3A00002C253032753A25303475004100492C01
:109F4A00253033692C253033692C253033692C258B
:109F5A003033692C253033690D0A002138204572C7
:109F6A00723A20556E6B6E6F776E20636F6D6D61FE
:109F7A006E642027256325633A25325825325827EF
:109F8A000D0A002138204572723A20556E6B6E6FA9
:109F9A00776E20636F6D6D616E64202725633A25A5
:109FAA003258270D0A002137204572723A20457827
:109FBA00747261207061726D617465720D0A00219C
:109FCA0036204572723A20496E76616C6964207057
:109FDA006172616D7465722076616C75650D0A0037
:109FEA002134204572723A204D697373696E672075
:109FFA00706172616D657465722873290D0A00219A
:10A00A0033204572723A205258204275666665724C
:10A01A00206F76657272756E0D0A002132204572C4
:10A02A00723A20545820427566666572206F7665CA
:10A03A007272756E0D0A002131204572723A204300
:10A04A00616E277420737465702074686174206669
:10A05A006173740D0A002130200D0A0020080025C2
:10A06A0073001B5B421B5B314B1B5B3047000401D7
:10A07A0030511F0B010801E012003051600BE84219
:10A08A00E842E842E842E842010801E0120034519D
:10A09A0003E0340501E012003151220A31E0030ADB
:10A0AA0024E0010A15E0210A0DE0010A01E012008C
:10A0BA000601A00EBD6F060EBE6F080EC06FC16B03
:10A0CA00BF8121D00601A00EBD6F060EBE6F1BD048
:10A0DA0036C4C5F637C4C6F60601800EC26F060E30
:10A0EA00C36FC76BC86BC48F12000601800EBD6FA9
:10A0FA00060EBE6F070EC06FC16BC10EBF6F120096
:10A10A0032C49BF60601BF8F12000601806B4B0E0C
:10A11A00816F826B836B846B856B080E866F8F6B86
:10A12A001A0EE66E010EE66E78EC42F0E552E55242
:10A13A001E0EE66E020EE66E78EC42F0E552E5522D
:10A14A002FD902E2E16AE5524FD90601996B9A6B5F
:10A15A00906B12001CD982D9050E3D1801E13E50C0
:10A16A0002E0000E18D051D9060197514B1808E1A8
:10A17A0098514C1805E114D902E2E16AE55234D942
:10A18A0044D9060199514B1805E19A514C1802E13C
:10A19A00906B956B010E0CD1FAD806018F6B975113
:10A1AA00981102E1000E05D045D9EF50800B01E06D
:10A1BA00010E000931E1FB0EDBCF4BF03BD9EE5229
:10A1CA00EF50D8804B5405E235D9EE52FB0EEFCF53
:10A1DA00DBFF8F6BFB0EDB508F5D19E28F51EA6A52
:10A1EA00400FE96E060EEA22EF50E66E8F51E76ED7
:10A1FA00FC0EDBCFE9FFFD0EDBCFEAFFE750E926D5
:10A20A00000EEA22E552E750EF6E8F2BE3D7C8D84B
:10A21A0002E2E16AE552E8D806018F51C9D0B7D8FF
:10A22A000601905107E1E7D8FB0EDBCF95F6010E48
:10A23A00966F906FBDD00BD917E1C0D8EDD802E167
:10A24A004C500BE0010EDBCFE9FFDB2A020EDBCF1D
:10A25A00EAFF01E3DB2AEF50F1E1CDD8DFCF95F633
:10A26A000601010E966F906FE552E552E552A0D0B5
:10A27A00EED818E1A3D8D0D802E14C500CE0010E78
:10A28A00DBCFF6FFDB2A020EDBCFF7FF01E3DB2A87
:10A29A000800F550F0E1AFD8DFCF95F60601966BCE
:10A2AA00010E906FE552E552E55282D070D8E6521F
:10A2BA00E652060199519A1102E1000E08D099C698
:10A2CA00E9FF9AC6EAFFEF50800B01E0010E000990
:10A2DA005BE1030E905D01E1906B905155E0020E37
:10A2EA00905D0DE1E66A000EE66EE66A8BD802E240
:10A2FA00E16AE55298D80601030E906F45D09005A1
:10A30A0043E1400E4B6E4C6A95514B5C000E4C5823
:10A31A0003E2400EDF6E02D095C6DFFFDF50955D87
:10A32A00956F000E936F060E946F010EDFCFDBFF61
:10A33A0096510BE1010EDB5012E091C6F6FF92C670
:10A34A00F7FF0800F55043D8F5D7010EDB5007E0B8
:10A35A0091C6E9FF92C6EAFFEF5039D8F6D706014F
:10A36A00955107E1400EDF5C02E1020E01D0030EB7
:10A37A00906FDFCFE6FF000EE66E060EE66E42D85D
:10A38A0002E2E16AE5524FD8E552E55211D0D9CF3F
:10A39A00E6FFDACFE6FFE1CFD9FFE2CFDAFF12001C
:10A3AA00400EE66E400EE66E060EE66EE66A47D090
:10A3BA00E552E5CFDAFFE7CFD9FF1200DF6A4ED8C0
:10A3CA00DE523DC0DEFF3EC0DDFFDD52120093C605
:10A3DA00E9FF94C6EAFFEF6E932B000E9423912BAC
:10A3EA009223010EDB061200E16E4B50F3CF97F673
:10A3FA00F4CF98F61200FC0EDBCF91F6FD0EDBCF00
:10A40A0092F61200010EE66E1AD0FA0EDBCF4BF06E
:10A41A00FB0EDBCF4CF01200DF2ADF504B6E4C6A8A
:10A42A00FF0E4B181200E16E4B50F3CF99F6F4CFA2
:10A43A009AF6120097C6E9FF98C6EAFF1200020EC2
:10A44A00E66E97EC42F04B6E050EE15C12009FDF60
:10A45A00E652E652E652060190511200FC0EDBCF9C
:10A46A003DF0FD0EDBCF3EF0120067D9E6520E0139
:10A47A00006BA96BDF6A180EDF5C14E280D9010E4B
:10A48A00E9260E0E82D9DF5074D9EF6A78D9490EBF
:10A49A00E9260E0E7AD973D9790EE9260E0E75D9E8
:10A4AA00DF2AE9D70E01C60EAC6F0E0EAD6F3F0E56
:10A4BA0079140009796ECF0E79140009796E7982C0
:10A4CA007B6A7A6A79900F0152815293F00EB41422
:10A4DA000909B46E0E01080EAA6F030EAB6F800E47
:10A4EA00AE6F3E0EAF6FE00EB06F2E0EB16F040E60
:10A4FA00B66F900EB26F010EB36F900EB46F010E6D
:10A50A00B56F000EE66EE66A010EE66E50EC3CF0A0
:10A51A00E552E552E552E55226D10FD9E652DF6AF5
:10A52A00180EDF5C0AE2DF5024D9EFCF4BF0FD0EA4
:10A53A00DB504B5C0AE0DF2AF3D7DF6A180EDF5CD8
:10A54A0008E2DF5016D9EF5002E1DF2803D0DF2AF4
:10A55A00F5D7000EE55207D1F0D8070EE12402E341
:10A56A00E168E652E16EDE6ADD6A020EDB6A030E1C
:10A57A00DB6A040EDB6A050EDB6A060EDB6A010E75
:10A58A00E66ED9CFE6FFDACFE6FF030EDFD8020F79
:10A59A0000D9010EDBD8030FFCD8030ED7D8050F5C
:10A5AA00F8D8030EFBD8295024E1020EDB50180814
:10A5BA0002E2298C1ED0050EDBCFE6FF060EDBCFAA
:10A5CA00E6FF030EDBCFE6FF040EDBCFE6FF020E4B
:10A5DA00DBCFE6FFDECFE6FFDDCFE6FF11D84B6E1D
:10A5EA00070EE15C02E2E16AE552E16E4B5055EC7E
:10A5FA002BF0070EE15C02E2E16AE552E16EB3D0AC
:10A60A009CD8E652E652FB0EDBCFE6FF86DFE55228
:10A61A00E76E010EE7CFDBFFDB5002E1000E8AD0C6
:10A62A00D950FC0FE96EFF0EDA20EA6EEE50ED10FB
:10A63A001FE1010EDB049DD8EF500E01EA6AAC253A
:10A64A00E96EAD51EA22EF6A86D8790EE9260E0E36
:10A65A009CD881D8490EE9260E0E97D8010EDB0444
:10A66A0088D8EF6A78D8010EE9260E0E8ED860D007
:10A67A00010EDB044B6E0E01AA514B5C59E2FB0E34
:10A68A00DB50180855E3FB0EDB50070802E1020114
:10A69A00F76B61D8010EE9260E0EEA22EE50ED1094
:10A6AA0010E1E66AFB0EDBCFE6FFF5EC32F0E5528D
:10A6BA00E552E66AFB0EDBCFE6FFC7EC32F0E55265
:10A6CA00E5521C50FEE00201030E846FF70EDBCF49
:10A6DA0092F2F80EDBCF93F2946B956B190E406EE3
:10A6EA00416A426A436A92C23BF093C23CF094C206
:10A6FA003DF095C23EF0F1EC55F037C092F238C009
:10A70A0093F239C094F23AC095F2010EDBCF99F276
:10A71A00FB0EDBCF98F2FC0EDBCF96F2FD0EDBCF01
:10A72A0097F2F90EDBCF9AF2FA0EDBCF9BF21C6A94
:10A73A00010EDB50E552E55216D0D9CFE6FFDACF4B
:10A74A00E6FFE1CFD9FFE2CFDAFF120027D8010EE8
:10A75A00E66ED9501200010EDB04E96EEA6AD8905F
:10A76A00E936EA361200E552E5CFDAFFE7CFD9FF3C
:10A77A001200EA6A310FE96E0E0EEA221200EA6A44
:10A78A00DF34FE0BEA36E96E1200EA22EE6AED6A5F
:10A79A001200E66E000EDA20E66E1200E66E98EC03
:10A7AA0030F0E552E552E552E552120005D8BAEC0E
:10A7BA0041F033EC27F0FBD78ED8E652E6520F0170
:10A7CA0048694969600ED36E9B8C580EDE6E020E84
:10A7DA00DD6EDFCF4BF0DF06010EDBCF4CF001E27E
:10A7EA00DB064B504C10F5E1948EA7EC26F050ECAA
:10A7FA0041F0E552E55278D0120012001200120020
:10A80A003CEF50F012008AEF50F00601CB051EE132
:10A81A000601CC051BE1F1DF65920601CC6B020152
:10A82A00100EF96F0E0EFA6FF907000EFA5BF95166
:10A83A00FA11FAE16584080EF96F070EFA6FF90743
:10A84A00000EFA5BF951FA11FAE16594120043D845
:10A85A00FC0EDBCF3DF0FD0EDBCF3EF0050E3D18C2
:10A86A0001E13E5036E0E8683D1802E17F0E3E18ED
:10A87A002FE0030E3D1801E13E5028E0020E3D187C
:10A88A0001E13E5021E0010E3D1801E13E501AE07F
:10A89A00740E3D1801E13E5013E0750E3D1801E1BA
:10A8AA003E500CE0730E3D1801E13E5005E0720E79
:10A8BA003D180FE13E500DD0A1DF0BD09DDF09D02E
:10A8CA009CDF07D0A0DF05D09DDF03D099DF01D040
:10A8DA0096DF010E09D0D9CFE6FFDACFE6FFE1CF46
:10A8EA00D9FFE2CFDAFF1200E552E5CFDAFFE7CF70
:10A8FA00D9FF12002A0EF66E100EF76E000EF86ED1
:10A90A0005010900F550E66F0900F550E76F03E10C
:10A91A00E66701D03DD00900F550E16F0900F55016
:10A92A00E26F0900F550E36F09000900F550E96E7E
:10A93A000900F550EA6E090009000900F550E46FB4
:10A94A000900F550E56F09000900F6CFE8F5F7CFE1
:10A95A00E9F5F8CFEAF5E1C5F6FFE2C5F7FFE3C589
:10A96A00F8FF0501E45302E1E55307E00900F55059
:10A97A00EE6EE407F8E2E507F9D7E8C5F6FFE9C5A0
:10A98A00F7FFEAC5F8FF0501E607000EE75BBFD748
:10A99A001200FE0EE3CFE9FFFF0EE3CFEAFFE9CF95
:10A9AA00F3FFEACFF4FFFB0EE35003E1FC0EE350A2
:10A9BA0009E0FB0EE30602E2FC0EE306FD0EE3509D
:10A9CA00EE6EF1D71200FE0EE3CFE9FFFF0EE3CFE2
:10A9DA00EAFFF36AF46AEE5203E0F34AF42AFBD779
:10A9EA001200FF0EE3CFF8FFE552FF0EE3CFF7FFA9
:10A9FA00E552FF0EE3CFF6FFE552E66AE66AE66A3B
:10AA0A000900F55209E0FD0EE32A05E1FE0EE32AEC
:10AA1A0002E1FF0EE32AF4D7FD0EE3CF3CF0FE0E6F
:10AA2A00E3CF3DF0FF0EE3CF3EF01200D9CFE6FFB1
:10AA3A00DACFE6FFE1CFD9FFE2CFDAFFE652E652FC
:10AA4A00E652E652D950FB0F4B6EFF0EDA204C6EDF
:10AA5A004BC0DEFFDD6EDECFE6FFDDCFE6FFFB0E8D
:10AA6A00DBCFE6FFFC0EDBCFE6FFFD0EDBCFE6FF1A
:10AA7A00FBC2E6FFFCC2E6FF2CEC48F04B6E070E69
:10AA8A00E15C02E2E16AE552E16E4B50020EF3CF5D
:10AA9A00DBFF030EF4CFDBFF020EDBCF4BF0030E1E
:10AAAA00DBCF4CF04BC0F3FF4CC0F4FF040EE15C6B
:10AABA0002E2E16AE552E16EE552E5CFDAFFE7CF5D
:10AACA00D9FF12001201000202000040D80492FDD0
:10AADA0082010102000109024300020100C0320999
:10AAEA0004000001020201000524001001042402EE
:10AAFA000205240600010524010001070581030857
:10AB0A00000209040100020A0000000705020240CF
:10AB1A0000000705820240000004030904180353D9
:10AB2A0000630068006D0061006C007A00480061F3
:10AB3A00007500730016034500690042006F007437
:10AB4A000042006F00610072006400E0AA23AB2794
:03AB5A00AB3FAB63
:10AB5E00D9CFE6FFDACFE6FFE1CFD9FFE2CFDAFFBA
:10AB6E00FB0EDBCF4BF0FC0EDBCF4CF00001800E6A
:10AB7E004C141AE1FB0EDBCFE9FFFC0EDBCFEAFF34
:10AB8E00EECFF3FFEDCFF4FFEE2A000EEF22F3CF60
:10AB9E00E9FFF4CFEAFFFD0EDBCFEFFFEF504C6A7B
:10ABAE00F36E4CC0F4FF10D0FB0EDB50FE0806E136
:10ABBE00FD0EDBCFE6FFD9EC56F005D0FD0EDBCF58
:10ABCE00E6FF9AEC28F0E552E552E5CFDAFFE7CF43
:10ABDE00D9FF12003B504002F3CF37F0F4CF38F0DC
:10ABEE004102F3503826000EF420396E3B504202DB
:10ABFE00F3503926000EF4203A6E3B504302F350C8
:10AC0E003A263C504002F3503826F4503922000EBA
:10AC1E003A223C504102F3503926F4503A223C502D
:10AC2E004202F3503A263D504002F3503926F4507A
:10AC3E003A223D504102F3503A263E504002F35024
:10AC4E003A2612003EC04AF03DC049F03D50420245
:10AC5E00F4CF3CF0F3CF3BF03E504302F4CF3EF046
:10AC6E00F3CF3DF04202F3503C26F4503D22E86A09
:10AC7E003E2249504302F3503C26F4503D22E86AEE
:10AC8E003E2243AE4FEF56F049503D5E4A503E5A7B
:10AC9E004AAE000C42503D5E43503E5A000CFF0E31
:10ACAE00E124E96EFF0EE220EA6EEDCFF4FFEFCF66
:10ACBE00F3FFF46607D0600EF36404D07B0EF360EE
:10ACCE0001D0F39A1200F36AF46AFF0EE124E96EE2
:10ACDE00FF0EE220EA6EED6607D02F0EEF6404D071
:10ACEE003A0EEF6001D0F32A12003A6A396A386AD6
:10ACFE00376A200EE76ED8903B363C363D363E36F0
:10AD0E003736383639363A364050375C4150385837
:10AD1E004250395843503A5809E34050375E41503B
:10AD2E00385A4250395A43503A5A3B2AE72EE4D702
:10AD3E0012004F4B0D0A000D0A0045424276313388
:10AD4E005F616E645F61626F766520454220466981
:10AD5E00726D776172652056657273696F6E2032FF
:07AD6E002E332E300D0A0008
:10AD7600C00EF36E00EE00F00E0E01D81200EA606F
:10AD860002D0EE6AFCD7F350E9601200EE6AFCD7F7
:10AD96001DEE00F02DEE00F0F86A469C7FEC54F0B4
:10ADA600FBEC56F0DBEC53F0FBD71200FF0EE35042
:10ADB600ADBA04D0B06AAC8EAD8A949CADA2FED773
:10ADC600AE6EF36EF46A1200F36AF46AF32A0F0B9E
:10ADD60005E0D890F336F436E804FBE11200303192
:0FADE6003233343536373839616263646566005D
:10ADF6001200FEFF0000000000000000000000003E
:10AE0600000000000000000000000000000000003C
:10AE1600000000000000000000000000000000002C
:10AE2600000000000000000000000000000000001C
:10AE3600000000000000000000000000000000000C
:10AE460000000000000000000000000000000000FC
:10AE56000000000000000000920F920F920F930F67
:10AE6600930F930F930F930F930F930F930F940FCB
:10AE7600940F940F940F940F940F940F940F950FB3
:10AE8600950F950F950F950F950F890F890F890FC0
:10AE96008A0F8A0F8A0F8A0F8A0F8A0F8A0F8A0FE4
:10AEA6008B0F8B0F8B0F8B0F8B0F8B0F8B0F8B0FCC
:10AEB6008C0F8C0F8C0F8C0F8C0F8C0F00010500E4
:10AEC6000102030405060700010203040506070242
:05AED60003040506075E
:08FFF800ACF70AFF63F801F009
:00000001FF
